BL51 BANKED LINKER/LOCATER V4.13                                                        04/17/2013  16:59:47  PAGE 1


BL51 BANKED LINKER/LOCATER V4.13, INVOKED BY:
C:\KEIL\C51\BIN\BL51.EXE ..\OBJ\main.obj, ..\OBJ\LCD drive.obj, ..\OBJ\Touch.obj TO ..\OBJ\LCD PRINT (.\LCD.m51) RAMSIZE
>>  (256)


MEMORY MODEL: SMALL


INPUT MODULES INCLUDED:
  ..\OBJ\main.obj (MAIN)
  ..\OBJ\LCD drive.obj (LCD_DRIVE)
  ..\OBJ\Touch.obj (TOUCH)
  C:\KEIL\C51\LIB\C51S.LIB (?C_STARTUP)
  C:\KEIL\C51\LIB\C51S.LIB (?C?COPY)
  C:\KEIL\C51\LIB\C51S.LIB (?C?UIDIV)


LINK MAP OF MODULE:  ..\OBJ\LCD (MAIN)


            TYPE    BASE      LENGTH    RELOCATION   SEGMENT NAME
            -----------------------------------------------------

            * * * * * * *   D A T A   M E M O R Y   * * * * * * *
            REG     0000H     0008H     ABSOLUTE     "REG BANK 0"
            DATA    0008H     0024H     UNIT         _DATA_GROUP_
            DATA    002CH     000AH     UNIT         ?DT?MAIN
            IDATA   0036H     0001H     UNIT         ?STACK

            * * * * * * *   C O D E   M E M O R Y   * * * * * * *
            CODE    0000H     0003H     ABSOLUTE     
            CODE    0003H     0003H     ABSOLUTE     
            CODE    0006H     229CH     UNIT         ?PR?LCD_INIT?LCD_DRIVE
            CODE    22A2H     066BH     UNIT         ?CO?LCD_DRIVE
            CODE    290DH     01CFH     UNIT         ?PR?_LCD_SETPOS?TOUCH
            CODE    2ADCH     014BH     UNIT         ?C?LIB_CODE
            CODE    2C27H     012CH     UNIT         ?PR?_LCD_TEST_SINGLECOLOR?LCD_DRIVE
            CODE    2D53H     0121H     UNIT         ?PR?MAIN?MAIN
            CODE    2E74H     00F9H     UNIT         ?PR?_LCD_SETWINDOW?LCD_DRIVE
            CODE    2F6DH     00C9H     UNIT         ?PR?_GUI_SPRINTF_CHAR?LCD_DRIVE
            CODE    3036H     00B7H     UNIT         ?PR?_LCD_ID_9341?LCD_DRIVE
            CODE    30EDH     00AEH     UNIT         ?PR?_LCD_ID?LCD_DRIVE
            CODE    319BH     008DH     UNIT         ?PR?_LCD_ID_61581?LCD_DRIVE
            CODE    3228H     0083H     UNIT         ?PR?MAKPIX?TOUCH
            CODE    32ABH     0078H     UNIT         ?PR?INRT?TOUCH
            CODE    3323H     0073H     UNIT         ?PR?_LCD_WRITE_DATA?LCD_DRIVE
            CODE    3396H     0062H     UNIT         ?PR?_LLCD_WRITE_CMD?LCD_DRIVE
            CODE    33F8H     004FH     UNIT         ?PR?_GUI_SPRINTF_STRING?LCD_DRIVE
            CODE    3447H     004AH     UNIT         ?PR?GETPIX?TOUCH
            CODE    3491H     0043H     UNIT         ?PR?_LLCD_WRITE_DATA?LCD_DRIVE
            CODE    34D4H     0041H     UNIT         ?PR?_DRAWPOINT?TOUCH
            CODE    3515H     0040H     UNIT         ?PR?_DELAYMS?LCD_DRIVE
            CODE    3555H     003BH     UNIT         ?PR?AD7843?TOUCH
            CODE    3590H     0032H     UNIT         ?PR?_LCD_WRITE_CMD?LCD_DRIVE
            CODE    35C2H     0030H     UNIT         ?PR?_UART_SEND_DATA?LCD_DRIVE
            CODE    35F2H     0026H     UNIT         ?PR?READFROMCHARFROM7843?TOUCH
            CODE    3618H     0025H     UNIT         ?PR?LCD_READ_8347ID?LCD_DRIVE
            CODE    363DH     0024H     UNIT         ?PR?LCD_READ_ID?LCD_DRIVE
BL51 BANKED LINKER/LOCATER V4.13                                                      04/17/2013  16:59:47  PAGE 2


            CODE    3661H     0021H     UNIT         ?PR?LCD_READ_ID9341?LCD_DRIVE
            CODE    3682H     001AH     UNIT         ?PR?LCD_READ_ID61581?LCD_DRIVE
            CODE    369CH     001AH     UNIT         ?PR?HD_RESET?LCD_DRIVE
            CODE    36B6H     0019H     UNIT         ?PR?_WRITECHARTO7843?TOUCH
            CODE    36CFH     0016H     UNIT         ?PR?_SENG_CMD_DAT?LCD_DRIVE
            CODE    36E5H     000FH     UNIT         ?PR?UART_INIT?LCD_DRIVE
            CODE    36F4H     000EH     UNIT         ?PR?_GUI_POINT?LCD_DRIVE
            CODE    3702H     000DH     UNIT         ?PR?KEYPRESS?LCD_DRIVE
            CODE    370FH     000CH     UNIT         ?PR?_DELAYUS?LCD_DRIVE
            CODE    371BH     000CH     UNIT         ?C_C51STARTUP
            CODE    3727H     000BH     UNIT         ?PR?_DELAY?TOUCH
            CODE    3732H     0009H     UNIT         ?PR?_LCD_SETXY?LCD_DRIVE
            CODE    373BH     0009H     UNIT         ?PR?SPISTART?TOUCH



OVERLAY MAP OF MODULE:   ..\OBJ\LCD (MAIN)


SEGMENT                                       DATA_GROUP 
  +--> CALLED SEGMENT                       START    LENGTH
-----------------------------------------------------------
?PR?INRT?TOUCH                              0008H    0004H
  +--> ?PR?_DELAY?TOUCH
  +--> ?PR?SPISTART?TOUCH
  +--> ?PR?_WRITECHARTO7843?TOUCH
  +--> ?PR?READFROMCHARFROM7843?TOUCH

*** NEW ROOT ***************************************************

?C_C51STARTUP                               -----    -----
  +--> ?PR?MAIN?MAIN

?PR?MAIN?MAIN                               000CH    0004H
  +--> ?PR?LCD_READ_ID9341?LCD_DRIVE
  +--> ?PR?LCD_READ_ID61581?LCD_DRIVE
  +--> ?PR?LCD_READ_ID?LCD_DRIVE
  +--> ?PR?LCD_READ_8347ID?LCD_DRIVE
  +--> ?PR?_DELAYMS?LCD_DRIVE
  +--> ?PR?LCD_INIT?LCD_DRIVE
  +--> ?PR?KEYPRESS?LCD_DRIVE
  +--> ?PR?_LCD_TEST_SINGLECOLOR?LCD_DRIVE
  +--> ?PR?SPISTART?TOUCH
  +--> ?PR?GETPIX?TOUCH
  +--> ?PR?_DRAWPOINT?TOUCH

?PR?LCD_READ_ID9341?LCD_DRIVE               -----    -----
  +--> ?PR?HD_RESET?LCD_DRIVE
  +--> ?PR?_DELAYMS?LCD_DRIVE
  +--> ?PR?_LCD_ID_9341?LCD_DRIVE
  +--> ?PR?_UART_SEND_DATA?LCD_DRIVE

?PR?HD_RESET?LCD_DRIVE                      -----    -----
  +--> ?PR?UART_INIT?LCD_DRIVE
  +--> ?PR?_DELAYMS?LCD_DRIVE

?PR?_DELAYMS?LCD_DRIVE                      0018H    0002H
BL51 BANKED LINKER/LOCATER V4.13                                                      04/17/2013  16:59:47  PAGE 3


  +--> ?PR?_UART_SEND_DATA?LCD_DRIVE
  +--> ?PR?_DELAYUS?LCD_DRIVE

?PR?_UART_SEND_DATA?LCD_DRIVE               -----    -----
  +--> ?PR?UART_INIT?LCD_DRIVE

?PR?_LCD_ID_9341?LCD_DRIVE                  0010H    0006H
  +--> ?PR?_LLCD_WRITE_CMD?LCD_DRIVE
  +--> ?PR?_DELAYMS?LCD_DRIVE
  +--> ?PR?_UART_SEND_DATA?LCD_DRIVE

?PR?_LLCD_WRITE_CMD?LCD_DRIVE               -----    -----
  +--> ?PR?_LLCD_WRITE_DATA?LCD_DRIVE

?PR?LCD_READ_ID61581?LCD_DRIVE              -----    -----
  +--> ?PR?HD_RESET?LCD_DRIVE
  +--> ?PR?_DELAYMS?LCD_DRIVE
  +--> ?PR?_LCD_ID_61581?LCD_DRIVE
  +--> ?PR?_UART_SEND_DATA?LCD_DRIVE

?PR?_LCD_ID_61581?LCD_DRIVE                 0010H    0008H
  +--> ?PR?_LLCD_WRITE_CMD?LCD_DRIVE
  +--> ?PR?_LLCD_WRITE_DATA?LCD_DRIVE
  +--> ?PR?_DELAYMS?LCD_DRIVE
  +--> ?PR?_UART_SEND_DATA?LCD_DRIVE

?PR?LCD_READ_ID?LCD_DRIVE                   -----    -----
  +--> ?PR?HD_RESET?LCD_DRIVE
  +--> ?PR?_DELAYMS?LCD_DRIVE
  +--> ?PR?_SENG_CMD_DAT?LCD_DRIVE
  +--> ?PR?_LCD_ID?LCD_DRIVE
  +--> ?PR?_UART_SEND_DATA?LCD_DRIVE

?PR?_SENG_CMD_DAT?LCD_DRIVE                 -----    -----
  +--> ?PR?_LLCD_WRITE_CMD?LCD_DRIVE
  +--> ?PR?_LLCD_WRITE_DATA?LCD_DRIVE

?PR?_LCD_ID?LCD_DRIVE                       0010H    0008H
  +--> ?PR?_LLCD_WRITE_CMD?LCD_DRIVE
  +--> ?PR?_DELAYMS?LCD_DRIVE

?PR?LCD_READ_8347ID?LCD_DRIVE               -----    -----
  +--> ?PR?HD_RESET?LCD_DRIVE
  +--> ?PR?_DELAYMS?LCD_DRIVE
  +--> ?PR?_SENG_CMD_DAT?LCD_DRIVE
  +--> ?PR?_LCD_ID?LCD_DRIVE
  +--> ?PR?_UART_SEND_DATA?LCD_DRIVE

?PR?LCD_INIT?LCD_DRIVE                      -----    -----
  +--> ?PR?_SENG_CMD_DAT?LCD_DRIVE
  +--> ?PR?_DELAYMS?LCD_DRIVE
  +--> ?PR?_LCD_TEST_SINGLECOLOR?LCD_DRIVE
  +--> ?CO?LCD_DRIVE
  +--> ?PR?_GUI_SPRINTF_STRING?LCD_DRIVE
  +--> ?PR?_LLCD_WRITE_CMD?LCD_DRIVE
  +--> ?PR?_LLCD_WRITE_DATA?LCD_DRIVE

BL51 BANKED LINKER/LOCATER V4.13                                                      04/17/2013  16:59:47  PAGE 4


?PR?_LCD_TEST_SINGLECOLOR?LCD_DRIVE         0010H    0003H
  +--> ?PR?_LCD_WRITE_DATA?LCD_DRIVE
  +--> ?PR?_LCD_WRITE_CMD?LCD_DRIVE
  +--> ?PR?_LLCD_WRITE_CMD?LCD_DRIVE

?PR?_LCD_WRITE_DATA?LCD_DRIVE               -----    -----
  +--> ?PR?_LCD_WRITE_CMD?LCD_DRIVE

?PR?_GUI_SPRINTF_STRING?LCD_DRIVE           0010H    0009H
  +--> ?CO?LCD_DRIVE
  +--> ?PR?_GUI_SPRINTF_CHAR?LCD_DRIVE

?PR?_GUI_SPRINTF_CHAR?LCD_DRIVE             0019H    000BH
  +--> ?CO?LCD_DRIVE
  +--> ?PR?_GUI_POINT?LCD_DRIVE

?PR?_GUI_POINT?LCD_DRIVE                    0024H    0002H
  +--> ?PR?_LCD_SETXY?LCD_DRIVE
  +--> ?PR?_LLCD_WRITE_DATA?LCD_DRIVE

?PR?_LCD_SETXY?LCD_DRIVE                    -----    -----
  +--> ?PR?_LCD_SETWINDOW?LCD_DRIVE

?PR?_LCD_SETWINDOW?LCD_DRIVE                0026H    0006H
  +--> ?PR?_SENG_CMD_DAT?LCD_DRIVE
  +--> ?PR?_LLCD_WRITE_CMD?LCD_DRIVE

?PR?KEYPRESS?LCD_DRIVE                      -----    -----
  +--> ?PR?_DELAYMS?LCD_DRIVE

?PR?GETPIX?TOUCH                            0010H    0008H
  +--> ?PR?AD7843?TOUCH
  +--> ?PR?MAKPIX?TOUCH

?PR?AD7843?TOUCH                            0018H    0004H
  +--> ?PR?_WRITECHARTO7843?TOUCH
  +--> ?PR?READFROMCHARFROM7843?TOUCH

?PR?MAKPIX?TOUCH                            0018H    0008H

?PR?_DRAWPOINT?TOUCH                        0010H    0004H
  +--> ?PR?_LCD_SETPOS?TOUCH
  +--> ?PR?_LLCD_WRITE_DATA?LCD_DRIVE

?PR?_LCD_SETPOS?TOUCH                       0014H    0008H
  +--> ?PR?_SENG_CMD_DAT?LCD_DRIVE
  +--> ?PR?_LLCD_WRITE_CMD?LCD_DRIVE
  +--> ?PR?_LLCD_WRITE_DATA?LCD_DRIVE



SYMBOL TABLE OF MODULE:  ..\OBJ\LCD (MAIN)

  VALUE           TYPE          NAME
  ----------------------------------

  -------         MODULE        MAIN
BL51 BANKED LINKER/LOCATER V4.13                                                      04/17/2013  16:59:47  PAGE 5


  C:0000H         SYMBOL        _ICE_DUMMY_
  D:0090H         PUBLIC        P1
  D:00B0H         PUBLIC        P3
  B:00B0H.4       PUBLIC        T0
  B:00D0H.6       PUBLIC        AC
  B:00B0H.5       PUBLIC        T1
  B:0090H.0       PUBLIC        T2
  B:00A8H.7       PUBLIC        EA
  D:002CH         PUBLIC        tempid
  D:00A8H         PUBLIC        IE
  B:00B0H.7       PUBLIC        CS
  B:00C8H.6       PUBLIC        EXF2
  B:00B0H.7       PUBLIC        RD
  B:00A8H.4       PUBLIC        ES
  D:00B8H         PUBLIC        IP
  B:0098H.0       PUBLIC        RI
  B:00B0H.2       PUBLIC        INT0
  B:00D0H.7       PUBLIC        CY
  B:0098H.1       PUBLIC        TI
  B:00B0H.3       PUBLIC        INT1
  B:00B0H.6       PUBLIC        DCLK
  B:00B8H.4       PUBLIC        PS
  B:0090H.1       PUBLIC        T2EX
  B:0090H.1       PUBLIC        RS
  B:00D0H.2       PUBLIC        OV
  C:2D53H         PUBLIC        main
  B:00C8H.1       PUBLIC        C_T2
  B:00B0H.6       PUBLIC        WR
  B:00C8H.5       PUBLIC        RCLK
  B:00C8H.4       PUBLIC        TCLK
  D:002EH         PUBLIC        zhiyi
  D:0098H         PUBLIC        SCON
  D:0088H         PUBLIC        TCON
  D:0030H         PUBLIC        temp
  B:00B0H.4       PUBLIC        DOUT
  B:0088H.1       PUBLIC        IE0
  B:0088H.3       PUBLIC        IE1
  B:00B0H.3       PUBLIC        BUSY
  B:00C8H.0       PUBLIC        CP_RL2
  B:00A8H.1       PUBLIC        ET0
  B:00A8H.3       PUBLIC        ET1
  B:0088H.5       PUBLIC        TF0
  B:00A8H.5       PUBLIC        ET2
  B:0088H.7       PUBLIC        TF1
  B:00C8H.7       PUBLIC        TF2
  B:0098H.2       PUBLIC        RB8
  B:00A8H.0       PUBLIC        EX0
  B:0088H.0       PUBLIC        IT0
  B:0098H.3       PUBLIC        TB8
  B:00A8H.2       PUBLIC        EX1
  B:0088H.2       PUBLIC        IT1
  B:00D0H.0       PUBLIC        P
  B:0098H.7       PUBLIC        SM0
  B:0098H.6       PUBLIC        SM1
  B:0098H.5       PUBLIC        SM2
  B:00B8H.1       PUBLIC        PT0
  B:00B8H.3       PUBLIC        PT1
BL51 BANKED LINKER/LOCATER V4.13                                                      04/17/2013  16:59:47  PAGE 6


  B:00D0H.3       PUBLIC        RS0
  B:00B8H.5       PUBLIC        PT2
  B:0088H.4       PUBLIC        TR0
  B:00D0H.4       PUBLIC        RS1
  B:0088H.6       PUBLIC        TR1
  B:0090H.3       PUBLIC        RDB
  B:00C8H.2       PUBLIC        TR2
  B:00B8H.0       PUBLIC        PX0
  B:00B8H.2       PUBLIC        PX1
  B:00B0H.5       PUBLIC        DIN
  B:00C8H.3       PUBLIC        EXEN2
  B:0090H.0       PUBLIC        TFT_CS
  B:0098H.4       PUBLIC        REN
  D:00C8H         PUBLIC        T2CON
  B:00B0H.3       PUBLIC        KEY
  B:0090H.4       PUBLIC        RES
  B:0090H.2       PUBLIC        WRB
  B:00B0H.0       PUBLIC        RXD
  B:00B0H.1       PUBLIC        TXD
  B:00B0H.3       PUBLIC        Penirq
  B:00D0H.5       PUBLIC        F0
  D:0032H         PUBLIC        Tp_pix
  D:00D0H         PUBLIC        PSW
  -------         PROC          MAIN
  -------         DO            MAIN
  D:0007H         SYMBOL        bawei
  D:000CH         SYMBOL        lx
  D:000EH         SYMBOL        ly
  -------         ENDDO         ly
  C:2D53H         LINE#         10
  C:2D53H         LINE#         11
  C:2D53H         LINE#         14
  C:2D58H         LINE#         16
  C:2D5BH         LINE#         17
  C:2D61H         LINE#         18
  C:2D61H         LINE#         19
  C:2D64H         LINE#         20
  C:2D64H         LINE#         23
  C:2D7CH         LINE#         24
  C:2D7CH         LINE#         25
  C:2D7FH         LINE#         26
  C:2D7FH         LINE#         29
  C:2D85H         LINE#         30
  C:2D85H         LINE#         31
  C:2D88H         LINE#         32
  C:2D90H         LINE#         33
  C:2D90H         LINE#         34
  C:2D96H         LINE#         35
  C:2D96H         LINE#         36
  C:2D96H         LINE#         37
  C:2D98H         LINE#         39
  C:2D9BH         LINE#         40
  C:2D9BH         LINE#         41
  C:2DA1H         LINE#         42
  C:2DA4H         LINE#         43
  C:2DA4H         LINE#         47
  C:2DABH         LINE#         48
BL51 BANKED LINKER/LOCATER V4.13                                                      04/17/2013  16:59:47  PAGE 7


  C:2DAEH         LINE#         50
  C:2DAEH         LINE#         51
  C:2DAEH         LINE#         53
  C:2DBAH         LINE#         54
  C:2DBAH         LINE#         56
  C:2DC6H         LINE#         57
  C:2DC6H         LINE#         58
  C:2DC9H         LINE#         59
  C:2DC9H         LINE#         66
  C:2DC9H         LINE#         68
  C:2DD1H         LINE#         69
  C:2DD1H         LINE#         71
  C:2DDDH         LINE#         72
  C:2DDDH         LINE#         73
  C:2DE0H         LINE#         74
  C:2DE0H         LINE#         79
  C:2DE6H         LINE#         80
  C:2DE9H         LINE#         81
  C:2DE9H         LINE#         82
  C:2DF0H         LINE#         84
  C:2DFCH         LINE#         85
  C:2DFCH         LINE#         86
  C:2DFFH         LINE#         87
  C:2DFFH         LINE#         95
  C:2E05H         LINE#         97
  C:2E11H         LINE#         98
  C:2E11H         LINE#         99
  C:2E14H         LINE#         100
  C:2E14H         LINE#         108
  C:2E1BH         LINE#         111
  C:2E27H         LINE#         112
  C:2E27H         LINE#         113
  C:2E2AH         LINE#         114
  C:2E2AH         LINE#         123
  C:2E2DH         LINE#         124
  C:2E2DH         LINE#         125
  C:2E2DH         LINE#         126
  C:2E30H         LINE#         127
  C:2E30H         LINE#         128
  C:2E36H         LINE#         129
  C:2E36H         LINE#         130
  C:2E51H         LINE#         131
  C:2E66H         LINE#         132
  C:2E72H         LINE#         133
  C:2E72H         LINE#         136
  -------         ENDPROC       MAIN
  -------         ENDMOD        MAIN

  -------         MODULE        LCD_DRIVE
  C:0000H         SYMBOL        _ICE_DUMMY_
  C:2E74H         PUBLIC        _LCD_setwindow
  D:0080H         PUBLIC        P0
  C:363DH         PUBLIC        LCD_read_id
  D:0090H         PUBLIC        P1
  D:00A0H         PUBLIC        P2
  D:00B0H         PUBLIC        P3
  B:00B0H.4       PUBLIC        T0
BL51 BANKED LINKER/LOCATER V4.13                                                      04/17/2013  16:59:47  PAGE 8


  B:00D0H.6       PUBLIC        AC
  B:00B0H.5       PUBLIC        T1
  B:0090H.0       PUBLIC        T2
  B:00A8H.7       PUBLIC        EA
  C:3682H         PUBLIC        LCD_read_id61581
  C:319BH         PUBLIC        _LCD_ID_61581
  D:00A8H         PUBLIC        IE
  C:36A4H         PUBLIC        HD_reset
  B:00C8H.6       PUBLIC        EXF2
  B:00B0H.7       PUBLIC        RD
  B:00A8H.4       PUBLIC        ES
  D:00B8H         PUBLIC        IP
  B:0098H.0       PUBLIC        RI
  B:00B0H.2       PUBLIC        INT0
  B:00D0H.7       PUBLIC        CY
  C:3364H         PUBLIC        _LCD_WRITE_DATA
  B:0098H.1       PUBLIC        TI
  B:00B0H.3       PUBLIC        INT1
  C:2C2BH         PUBLIC        _LCD_TEST_SingleColor
  C:30EDH         PUBLIC        _LCD_ID
  C:33B8H         PUBLIC        _LLCD_WRITE_CMD
  B:00B8H.4       PUBLIC        PS
  B:0090H.1       PUBLIC        T2EX
  B:0090H.1       PUBLIC        RS
  B:00D0H.2       PUBLIC        OV
  C:35EAH         PUBLIC        _UART_send_data
  B:00C8H.1       PUBLIC        C_T2
  B:00B0H.6       PUBLIC        WR
  C:340CH         PUBLIC        _GUI_sprintf_string
  B:00C8H.5       PUBLIC        RCLK
  B:00C8H.4       PUBLIC        TCLK
  D:0099H         PUBLIC        SBUF
  C:2F6DH         PUBLIC        _GUI_sprintf_char
  C:36F4H         PUBLIC        _GUI_Point
  D:0098H         PUBLIC        SCON
  D:0089H         PUBLIC        TMOD
  D:0088H         PUBLIC        TCON
  B:0088H.1       PUBLIC        IE0
  B:0088H.3       PUBLIC        IE1
  C:36D7H         PUBLIC        _seng_cmd_dat
  B:00C8H.0       PUBLIC        CP_RL2
  B:00A8H.1       PUBLIC        ET0
  B:00A8H.3       PUBLIC        ET1
  B:0088H.5       PUBLIC        TF0
  B:00A8H.5       PUBLIC        ET2
  B:0088H.7       PUBLIC        TF1
  B:00C8H.7       PUBLIC        TF2
  B:0098H.2       PUBLIC        RB8
  B:00A8H.0       PUBLIC        EX0
  B:0088H.0       PUBLIC        IT0
  D:008DH         PUBLIC        TH1
  B:0098H.3       PUBLIC        TB8
  B:00A8H.2       PUBLIC        EX1
  B:0088H.2       PUBLIC        IT1
  B:00D0H.0       PUBLIC        P
  B:0098H.7       PUBLIC        SM0
  B:0098H.6       PUBLIC        SM1
BL51 BANKED LINKER/LOCATER V4.13                                                      04/17/2013  16:59:47  PAGE 9


  D:008BH         PUBLIC        TL1
  C:231DH         PUBLIC        font16x8
  B:0098H.5       PUBLIC        SM2
  C:3539H         PUBLIC        _delayms
  C:3661H         PUBLIC        LCD_read_id9341
  C:3036H         PUBLIC        _LCD_ID_9341
  C:3732H         PUBLIC        _LCD_setxy
  C:36E5H         PUBLIC        UART_init
  B:00B8H.1       PUBLIC        PT0
  B:00B8H.3       PUBLIC        PT1
  B:00D0H.3       PUBLIC        RS0
  C:3590H         PUBLIC        _LCD_WRITE_CMD
  B:00B8H.5       PUBLIC        PT2
  B:0088H.4       PUBLIC        TR0
  B:00D0H.4       PUBLIC        RS1
  B:0088H.6       PUBLIC        TR1
  C:3618H         PUBLIC        LCD_read_8347id
  B:0090H.3       PUBLIC        RDB
  B:00C8H.2       PUBLIC        TR2
  B:00B8H.0       PUBLIC        PX0
  B:00B8H.2       PUBLIC        PX1
  C:370FH         PUBLIC        _delayus
  C:3702H         PUBLIC        Keypress
  B:00C8H.3       PUBLIC        EXEN2
  B:0090H.0       PUBLIC        TFT_CS
  B:0098H.4       PUBLIC        REN
  D:00C8H         PUBLIC        T2CON
  C:3494H         PUBLIC        _LLCD_WRITE_DATA
  B:00B0H.3       PUBLIC        KEY
  C:0006H         PUBLIC        LCD_init
  B:0090H.4       PUBLIC        RES
  B:0090H.2       PUBLIC        WRB
  B:00B0H.0       PUBLIC        RXD
  B:00B0H.1       PUBLIC        TXD
  B:00D0H.5       PUBLIC        F0
  D:00D0H         PUBLIC        PSW
  -------         PROC          UART_INIT
  C:36E5H         LINE#         8
  C:36E5H         LINE#         9
  C:36E5H         LINE#         10
  C:36E8H         LINE#         11
  C:36EBH         LINE#         12
  C:36EEH         LINE#         13
  C:36F1H         LINE#         14
  C:36F3H         LINE#         16
  -------         ENDPROC       UART_INIT
  C:35CBH         SYMBOL        L?0190
  -------         PROC          L?0189
  -------         ENDPROC       L?0189
  C:35CBH         SYMBOL        L?0190
  -------         PROC          _UART_SEND_DATA
  D:0007H         SYMBOL        lcdid
  C:35EAH         LINE#         21
  C:35EAH         LINE#         22
  C:35EAH         LINE#         24
  C:35ECH         LINE#         25
  C:35EFH         LINE#         26
BL51 BANKED LINKER/LOCATER V4.13                                                      04/17/2013  16:59:47  PAGE 10


  C:35F1H         LINE#         28
  -------         ENDPROC       _UART_SEND_DATA
  -------         PROC          LCD_INIT
  C:0006H         LINE#         33
  C:0006H         LINE#         34
  C:0006H         LINE#         36
  C:0015H         LINE#         37
  C:0015H         LINE#         38
  C:001EH         LINE#         39
  C:0029H         LINE#         40
  C:0034H         LINE#         45
  C:003DH         LINE#         46
  C:0048H         LINE#         47
  C:0051H         LINE#         48
  C:005AH         LINE#         49
  C:0063H         LINE#         50
  C:006CH         LINE#         51
  C:0075H         LINE#         52
  C:007CH         LINE#         54
  C:0087H         LINE#         55
  C:0092H         LINE#         56
  C:009DH         LINE#         57
  C:00A8H         LINE#         58
  C:00B3H         LINE#         59
  C:00BEH         LINE#         60
  C:00C9H         LINE#         61
  C:00D2H         LINE#         62
  C:00DBH         LINE#         63
  C:00E6H         LINE#         64
  C:00EFH         LINE#         65
  C:00FAH         LINE#         66
  C:0105H         LINE#         68
  C:0110H         LINE#         69
  C:0119H         LINE#         70
  C:0122H         LINE#         71
  C:012BH         LINE#         72
  C:0134H         LINE#         73
  C:013DH         LINE#         74
  C:0146H         LINE#         75
  C:014FH         LINE#         76
  C:015AH         LINE#         77
  C:0163H         LINE#         78
  C:016EH         LINE#         79
  C:0179H         LINE#         80
  C:0180H         LINE#         81
  C:0187H         LINE#         82
  C:018AH         LINE#         83
  C:01A1H         LINE#         84
  C:01A9H         LINE#         85
  C:01A9H         LINE#         86
  C:01B0H         LINE#         87
  C:01B0H         LINE#         88
  C:01B0H         LINE#         89
  C:01B3H         LINE#         90
  C:01B3H         LINE#         91
  C:01C2H         LINE#         92
  C:01C2H         LINE#         93
BL51 BANKED LINKER/LOCATER V4.13                                                      04/17/2013  16:59:47  PAGE 11


  C:01C8H         LINE#         94
  C:01CBH         LINE#         95
  C:01D2H         LINE#         96
  C:01D9H         LINE#         97
  C:01E0H         LINE#         98
  C:01E7H         LINE#         99
  C:01EEH         LINE#         100
  C:01F5H         LINE#         101
  C:01FCH         LINE#         102
  C:0203H         LINE#         103
  C:020AH         LINE#         104
  C:0211H         LINE#         105
  C:0218H         LINE#         106
  C:021FH         LINE#         107
  C:0226H         LINE#         108
  C:022DH         LINE#         109
  C:0230H         LINE#         110
  C:0237H         LINE#         111
  C:023EH         LINE#         112
  C:0245H         LINE#         113
  C:024CH         LINE#         114
  C:0253H         LINE#         115
  C:0259H         LINE#         116
  C:025FH         LINE#         117
  C:0266H         LINE#         118
  C:026DH         LINE#         119
  C:0274H         LINE#         120
  C:027BH         LINE#         121
  C:0282H         LINE#         122
  C:0289H         LINE#         123
  C:0290H         LINE#         124
  C:0297H         LINE#         125
  C:029EH         LINE#         126
  C:02A5H         LINE#         127
  C:02ACH         LINE#         128
  C:02B3H         LINE#         129
  C:02BAH         LINE#         130
  C:02C1H         LINE#         131
  C:02C7H         LINE#         132
  C:02CEH         LINE#         133
  C:02D5H         LINE#         134
  C:02DCH         LINE#         135
  C:02E3H         LINE#         136
  C:02EAH         LINE#         137
  C:02F0H         LINE#         138
  C:02F7H         LINE#         139
  C:02FEH         LINE#         140
  C:0305H         LINE#         141
  C:030CH         LINE#         142
  C:0313H         LINE#         143
  C:031AH         LINE#         144
  C:0321H         LINE#         145
  C:0328H         LINE#         146
  C:032FH         LINE#         147
  C:0336H         LINE#         148
  C:033DH         LINE#         149
  C:0344H         LINE#         150
BL51 BANKED LINKER/LOCATER V4.13                                                      04/17/2013  16:59:47  PAGE 12


  C:034BH         LINE#         151
  C:0352H         LINE#         152
  C:0358H         LINE#         153
  C:035EH         LINE#         154
  C:0364H         LINE#         155
  C:036AH         LINE#         156
  C:0371H         LINE#         157
  C:0377H         LINE#         158
  C:037EH         LINE#         159
  C:0385H         LINE#         160
  C:038CH         LINE#         161
  C:0393H         LINE#         162
  C:039AH         LINE#         163
  C:03A1H         LINE#         164
  C:03A8H         LINE#         165
  C:03AFH         LINE#         166
  C:03B6H         LINE#         167
  C:03BDH         LINE#         168
  C:03C4H         LINE#         169
  C:03CBH         LINE#         170
  C:03D2H         LINE#         171
  C:03D9H         LINE#         172
  C:03E0H         LINE#         173
  C:03E6H         LINE#         174
  C:03ECH         LINE#         175
  C:03F3H         LINE#         176
  C:03FAH         LINE#         177
  C:0401H         LINE#         178
  C:0407H         LINE#         179
  C:040DH         LINE#         180
  C:0413H         LINE#         181
  C:041AH         LINE#         182
  C:0421H         LINE#         183
  C:0428H         LINE#         184
  C:042FH         LINE#         185
  C:0432H         LINE#         186
  C:0449H         LINE#         187
  C:0451H         LINE#         188
  C:0451H         LINE#         189
  C:0458H         LINE#         190
  C:0458H         LINE#         191
  C:0458H         LINE#         192
  C:045BH         LINE#         193
  C:045BH         LINE#         194
  C:045BH         LINE#         195
  C:046AH         LINE#         196
  C:046AH         LINE#         197
  C:0470H         LINE#         198
  C:0479H         LINE#         199
  C:0482H         LINE#         200
  C:048BH         LINE#         201
  C:0492H         LINE#         204
  C:049DH         LINE#         205
  C:04A6H         LINE#         206
  C:04B1H         LINE#         207
  C:04BCH         LINE#         208
  C:04C7H         LINE#         210
BL51 BANKED LINKER/LOCATER V4.13                                                      04/17/2013  16:59:47  PAGE 13


  C:04D2H         LINE#         211
  C:04DDH         LINE#         212
  C:04E4H         LINE#         214
  C:04EFH         LINE#         215
  C:04FAH         LINE#         216
  C:0501H         LINE#         219
  C:050CH         LINE#         220
  C:0517H         LINE#         221
  C:0522H         LINE#         222
  C:052DH         LINE#         223
  C:0538H         LINE#         224
  C:0543H         LINE#         225
  C:054EH         LINE#         226
  C:0559H         LINE#         227
  C:0564H         LINE#         228
  C:056FH         LINE#         229
  C:057AH         LINE#         230
  C:0585H         LINE#         231
  C:058CH         LINE#         234
  C:0597H         LINE#         235
  C:05A2H         LINE#         236
  C:05ADH         LINE#         237
  C:05B6H         LINE#         238
  C:05C1H         LINE#         239
  C:05CCH         LINE#         240
  C:05D7H         LINE#         241
  C:05E0H         LINE#         242
  C:05EBH         LINE#         243
  C:05F4H         LINE#         244
  C:05FFH         LINE#         245
  C:0608H         LINE#         246
  C:0613H         LINE#         247
  C:061EH         LINE#         248
  C:0629H         LINE#         249
  C:0632H         LINE#         250
  C:0639H         LINE#         253
  C:063CH         LINE#         254
  C:0641H         LINE#         255
  C:0646H         LINE#         256
  C:064DH         LINE#         258
  C:0654H         LINE#         260
  C:0657H         LINE#         261
  C:066EH         LINE#         262
  C:0676H         LINE#         263
  C:0676H         LINE#         264
  C:067DH         LINE#         265
  C:067DH         LINE#         266
  C:067DH         LINE#         267
  C:0680H         LINE#         268
  C:0680H         LINE#         269
  C:0680H         LINE#         270
  C:068FH         LINE#         271
  C:068FH         LINE#         273
  C:0698H         LINE#         274
  C:06A2H         LINE#         275
  C:06A9H         LINE#         276
  C:06B4H         LINE#         277
BL51 BANKED LINKER/LOCATER V4.13                                                      04/17/2013  16:59:47  PAGE 14


  C:06BFH         LINE#         278
  C:06CAH         LINE#         279
  C:06D3H         LINE#         280
  C:06DEH         LINE#         281
  C:06E7H         LINE#         282
  C:06F0H         LINE#         283
  C:06F9H         LINE#         284
  C:0702H         LINE#         285
  C:070BH         LINE#         287
  C:0714H         LINE#         288
  C:071DH         LINE#         289
  C:0726H         LINE#         290
  C:072FH         LINE#         291
  C:0736H         LINE#         292
  C:0741H         LINE#         293
  C:074CH         LINE#         294
  C:0753H         LINE#         295
  C:075EH         LINE#         296
  C:0765H         LINE#         297
  C:0770H         LINE#         298
  C:077BH         LINE#         299
  C:0782H         LINE#         300
  C:078BH         LINE#         301
  C:0794H         LINE#         303
  C:079FH         LINE#         304
  C:07AAH         LINE#         305
  C:07B5H         LINE#         308
  C:07C0H         LINE#         309
  C:07CBH         LINE#         310
  C:07D6H         LINE#         311
  C:07E1H         LINE#         312
  C:07ECH         LINE#         313
  C:07F7H         LINE#         314
  C:0802H         LINE#         316
  C:080BH         LINE#         317
  C:0816H         LINE#         318
  C:081FH         LINE#         319
  C:082AH         LINE#         320
  C:0835H         LINE#         321
  C:0840H         LINE#         322
  C:0849H         LINE#         324
  C:0854H         LINE#         325
  C:085DH         LINE#         326
  C:0868H         LINE#         327
  C:0873H         LINE#         328
  C:087CH         LINE#         329
  C:0885H         LINE#         331
  C:088AH         LINE#         332
  C:0891H         LINE#         333
  C:0896H         LINE#         334
  C:089DH         LINE#         335
  C:08A4H         LINE#         336
  C:08ABH         LINE#         338
  C:08AEH         LINE#         339
  C:08C5H         LINE#         340
  C:08CDH         LINE#         341
  C:08CDH         LINE#         342
BL51 BANKED LINKER/LOCATER V4.13                                                      04/17/2013  16:59:47  PAGE 15


  C:08D4H         LINE#         343
  C:08D4H         LINE#         344
  C:08D4H         LINE#         345
  C:08D7H         LINE#         346
  C:08D7H         LINE#         347
  C:08D7H         LINE#         348
  C:08E6H         LINE#         349
  C:08E6H         LINE#         350
  C:08F1H         LINE#         351
  C:08FFH         LINE#         352
  C:090BH         LINE#         353
  C:0919H         LINE#         354
  C:0927H         LINE#         355
  C:0935H         LINE#         356
  C:0943H         LINE#         357
  C:0951H         LINE#         358
  C:095DH         LINE#         359
  C:096BH         LINE#         360
  C:0977H         LINE#         361
  C:0983H         LINE#         362
  C:0991H         LINE#         363
  C:099FH         LINE#         364
  C:09A9H         LINE#         365
  C:09B5H         LINE#         366
  C:09C1H         LINE#         367
  C:09CDH         LINE#         368
  C:09D9H         LINE#         369
  C:09E5H         LINE#         370
  C:09F3H         LINE#         371
  C:09FFH         LINE#         372
  C:0A0BH         LINE#         373
  C:0A19H         LINE#         374
  C:0A25H         LINE#         375
  C:0A33H         LINE#         376
  C:0A41H         LINE#         377
  C:0A4FH         LINE#         378
  C:0A5DH         LINE#         379
  C:0A6BH         LINE#         380
  C:0A79H         LINE#         381
  C:0A87H         LINE#         382
  C:0A95H         LINE#         383
  C:0AA3H         LINE#         384
  C:0AB1H         LINE#         385
  C:0ABFH         LINE#         386
  C:0ACBH         LINE#         387
  C:0AD7H         LINE#         388
  C:0AE5H         LINE#         389
  C:0AE8H         LINE#         390
  C:0AFFH         LINE#         391
  C:0B07H         LINE#         392
  C:0B07H         LINE#         393
  C:0B0EH         LINE#         394
  C:0B0EH         LINE#         395
  C:0B0EH         LINE#         396
  C:0B11H         LINE#         397
  C:0B11H         LINE#         398
  C:0B20H         LINE#         399
BL51 BANKED LINKER/LOCATER V4.13                                                      04/17/2013  16:59:47  PAGE 16


  C:0B20H         LINE#         400
  C:0B2AH         LINE#         401
  C:0B35H         LINE#         402
  C:0B40H         LINE#         403
  C:0B4BH         LINE#         404
  C:0B54H         LINE#         405
  C:0B5FH         LINE#         406
  C:0B68H         LINE#         407
  C:0B71H         LINE#         408
  C:0B7AH         LINE#         409
  C:0B83H         LINE#         410
  C:0B8CH         LINE#         412
  C:0B95H         LINE#         413
  C:0BA0H         LINE#         414
  C:0BA9H         LINE#         415
  C:0BB2H         LINE#         416
  C:0BBBH         LINE#         418
  C:0BC6H         LINE#         419
  C:0BD1H         LINE#         422
  C:0BDCH         LINE#         425
  C:0BE7H         LINE#         428
  C:0BF2H         LINE#         429
  C:0BFDH         LINE#         431
  C:0C08H         LINE#         432
  C:0C13H         LINE#         433
  C:0C1EH         LINE#         434
  C:0C29H         LINE#         435
  C:0C34H         LINE#         436
  C:0C3FH         LINE#         437
  C:0C4AH         LINE#         438
  C:0C55H         LINE#         439
  C:0C60H         LINE#         440
  C:0C6BH         LINE#         442
  C:0C74H         LINE#         443
  C:0C7FH         LINE#         444
  C:0C88H         LINE#         445
  C:0C93H         LINE#         446
  C:0C9EH         LINE#         447
  C:0CA9H         LINE#         448
  C:0CB2H         LINE#         450
  C:0CBBH         LINE#         451
  C:0CC4H         LINE#         452
  C:0CCDH         LINE#         453
  C:0CD6H         LINE#         454
  C:0CDFH         LINE#         455
  C:0CE8H         LINE#         457
  C:0CF3H         LINE#         458
  C:0CFEH         LINE#         460
  C:0D05H         LINE#         461
  C:0D0FH         LINE#         462
  C:0D12H         LINE#         463
  C:0D29H         LINE#         464
  C:0D31H         LINE#         465
  C:0D31H         LINE#         466
  C:0D38H         LINE#         467
  C:0D38H         LINE#         468
  C:0D38H         LINE#         469
BL51 BANKED LINKER/LOCATER V4.13                                                      04/17/2013  16:59:47  PAGE 17


  C:0D3BH         LINE#         470
  C:0D3BH         LINE#         471
  C:0D4AH         LINE#         472
  C:0D4AH         LINE#         473
  C:0D54H         LINE#         474
  C:0D5FH         LINE#         477
  C:0D6AH         LINE#         478
  C:0D75H         LINE#         479
  C:0D80H         LINE#         480
  C:0D89H         LINE#         481
  C:0D94H         LINE#         482
  C:0D9DH         LINE#         483
  C:0DA6H         LINE#         484
  C:0DB1H         LINE#         485
  C:0DBAH         LINE#         486
  C:0DC3H         LINE#         488
  C:0DCCH         LINE#         489
  C:0DD7H         LINE#         490
  C:0DE0H         LINE#         491
  C:0DE9H         LINE#         492
  C:0DECH         LINE#         493
  C:0DF3H         LINE#         494
  C:0DFEH         LINE#         495
  C:0E09H         LINE#         496
  C:0E10H         LINE#         497
  C:0E1BH         LINE#         498
  C:0E22H         LINE#         499
  C:0E2DH         LINE#         500
  C:0E38H         LINE#         501
  C:0E43H         LINE#         502
  C:0E4AH         LINE#         503
  C:0E53H         LINE#         504
  C:0E5CH         LINE#         505
  C:0E63H         LINE#         507
  C:0E6CH         LINE#         508
  C:0E77H         LINE#         509
  C:0E82H         LINE#         510
  C:0E8BH         LINE#         511
  C:0E96H         LINE#         512
  C:0EA1H         LINE#         513
  C:0EACH         LINE#         514
  C:0EB7H         LINE#         515
  C:0EC0H         LINE#         516
  C:0ECBH         LINE#         517
  C:0ED2H         LINE#         518
  C:0EDBH         LINE#         519
  C:0EE6H         LINE#         520
  C:0EEFH         LINE#         521
  C:0EFAH         LINE#         523
  C:0F05H         LINE#         524
  C:0F10H         LINE#         525
  C:0F19H         LINE#         526
  C:0F22H         LINE#         527
  C:0F2BH         LINE#         528
  C:0F34H         LINE#         529
  C:0F3DH         LINE#         530
  C:0F46H         LINE#         531
BL51 BANKED LINKER/LOCATER V4.13                                                      04/17/2013  16:59:47  PAGE 18


  C:0F4FH         LINE#         533
  C:0F5AH         LINE#         534
  C:0F65H         LINE#         536
  C:0F6CH         LINE#         537
  C:0F6FH         LINE#         538
  C:0F86H         LINE#         539
  C:0F8EH         LINE#         540
  C:0F8EH         LINE#         541
  C:0F95H         LINE#         542
  C:0F95H         LINE#         543
  C:0F95H         LINE#         544
  C:0F98H         LINE#         545
  C:0F98H         LINE#         546
  C:0FA7H         LINE#         547
  C:0FA7H         LINE#         548
  C:0FB1H         LINE#         549
  C:0FBCH         LINE#         550
  C:0FC7H         LINE#         551
  C:0FD2H         LINE#         553
  C:0FDDH         LINE#         554
  C:0FE6H         LINE#         555
  C:0FEFH         LINE#         556
  C:0FF8H         LINE#         557
  C:1001H         LINE#         558
  C:100AH         LINE#         560
  C:1013H         LINE#         561
  C:101EH         LINE#         562
  C:1027H         LINE#         563
  C:1030H         LINE#         564
  C:1037H         LINE#         565
  C:1042H         LINE#         566
  C:104DH         LINE#         567
  C:1054H         LINE#         568
  C:105FH         LINE#         569
  C:1066H         LINE#         570
  C:1071H         LINE#         571
  C:107CH         LINE#         572
  C:1087H         LINE#         573
  C:108EH         LINE#         574
  C:1097H         LINE#         575
  C:10A2H         LINE#         577
  C:10ABH         LINE#         578
  C:10B6H         LINE#         579
  C:10BFH         LINE#         580
  C:10CAH         LINE#         581
  C:10D5H         LINE#         582
  C:10E0H         LINE#         583
  C:10EBH         LINE#         584
  C:10F6H         LINE#         585
  C:1101H         LINE#         586
  C:110CH         LINE#         588
  C:1115H         LINE#         589
  C:1120H         LINE#         590
  C:1129H         LINE#         591
  C:1134H         LINE#         592
  C:113FH         LINE#         593
  C:114AH         LINE#         594
BL51 BANKED LINKER/LOCATER V4.13                                                      04/17/2013  16:59:47  PAGE 19


  C:1153H         LINE#         596
  C:115CH         LINE#         597
  C:1165H         LINE#         598
  C:116EH         LINE#         599
  C:1177H         LINE#         600
  C:1180H         LINE#         601
  C:1189H         LINE#         603
  C:1194H         LINE#         604
  C:119FH         LINE#         605
  C:11A6H         LINE#         606
  C:11A9H         LINE#         607
  C:11C0H         LINE#         608
  C:11C8H         LINE#         609
  C:11C8H         LINE#         610
  C:11CFH         LINE#         611
  C:11CFH         LINE#         612
  C:11CFH         LINE#         613
  C:11D2H         LINE#         614
  C:11D2H         LINE#         615
  C:11E1H         LINE#         616
  C:11E1H         LINE#         618
  C:11E9H         LINE#         619
  C:11F0H         LINE#         620
  C:11FBH         LINE#         621
  C:1206H         LINE#         622
  C:1211H         LINE#         623
  C:121CH         LINE#         624
  C:1227H         LINE#         626
  C:1232H         LINE#         627
  C:123DH         LINE#         628
  C:1248H         LINE#         629
  C:1253H         LINE#         630
  C:125EH         LINE#         631
  C:1269H         LINE#         632
  C:1274H         LINE#         633
  C:127FH         LINE#         634
  C:1288H         LINE#         635
  C:1291H         LINE#         636
  C:129CH         LINE#         637
  C:12A5H         LINE#         638
  C:12B0H         LINE#         639
  C:12B9H         LINE#         640
  C:12C0H         LINE#         641
  C:12C3H         LINE#         642
  C:12CEH         LINE#         643
  C:12D5H         LINE#         645
  C:12E0H         LINE#         646
  C:12EBH         LINE#         647
  C:12F6H         LINE#         648
  C:1301H         LINE#         649
  C:130AH         LINE#         650
  C:1315H         LINE#         651
  C:1320H         LINE#         653
  C:1329H         LINE#         654
  C:1334H         LINE#         655
  C:133DH         LINE#         656
  C:1348H         LINE#         658
BL51 BANKED LINKER/LOCATER V4.13                                                      04/17/2013  16:59:47  PAGE 20


  C:1353H         LINE#         659
  C:135EH         LINE#         660
  C:1367H         LINE#         661
  C:1370H         LINE#         663
  C:1379H         LINE#         664
  C:1382H         LINE#         665
  C:138BH         LINE#         666
  C:1394H         LINE#         667
  C:139DH         LINE#         669
  C:13A8H         LINE#         670
  C:13B3H         LINE#         671
  C:13BEH         LINE#         672
  C:13C7H         LINE#         673
  C:13D0H         LINE#         674
  C:13D9H         LINE#         676
  C:13E4H         LINE#         677
  C:13EFH         LINE#         678
  C:13FAH         LINE#         679
  C:1403H         LINE#         680
  C:140CH         LINE#         681
  C:1415H         LINE#         682
  C:141EH         LINE#         683
  C:1427H         LINE#         684
  C:142CH         LINE#         685
  C:1433H         LINE#         686
  C:1438H         LINE#         687
  C:143FH         LINE#         688
  C:1446H         LINE#         689
  C:144DH         LINE#         690
  C:1450H         LINE#         691
  C:1467H         LINE#         692
  C:146FH         LINE#         693
  C:146FH         LINE#         694
  C:1476H         LINE#         695
  C:1476H         LINE#         696
  C:1476H         LINE#         697
  C:1479H         LINE#         698
  C:1479H         LINE#         699
  C:1488H         LINE#         700
  C:1488H         LINE#         701
  C:148FH         LINE#         702
  C:1497H         LINE#         703
  C:149FH         LINE#         704
  C:14A7H         LINE#         706
  C:14B2H         LINE#         707
  C:14B9H         LINE#         708
  C:14C4H         LINE#         709
  C:14CFH         LINE#         711
  C:14DAH         LINE#         712
  C:14E5H         LINE#         713
  C:14F0H         LINE#         714
  C:14FBH         LINE#         715
  C:1506H         LINE#         716
  C:1511H         LINE#         717
  C:151CH         LINE#         718
  C:1527H         LINE#         719
  C:1532H         LINE#         720
BL51 BANKED LINKER/LOCATER V4.13                                                      04/17/2013  16:59:47  PAGE 21


  C:153DH         LINE#         722
  C:1548H         LINE#         723
  C:1551H         LINE#         724
  C:155CH         LINE#         725
  C:1565H         LINE#         726
  C:156EH         LINE#         727
  C:1575H         LINE#         729
  C:1580H         LINE#         730
  C:158BH         LINE#         731
  C:1592H         LINE#         733
  C:159DH         LINE#         734
  C:15A4H         LINE#         736
  C:15AFH         LINE#         737
  C:15BAH         LINE#         738
  C:15C5H         LINE#         739
  C:15CCH         LINE#         741
  C:15D7H         LINE#         742
  C:15E2H         LINE#         743
  C:15EDH         LINE#         744
  C:15F8H         LINE#         745
  C:1601H         LINE#         746
  C:160AH         LINE#         747
  C:1613H         LINE#         748
  C:161EH         LINE#         749
  C:1627H         LINE#         750
  C:1632H         LINE#         751
  C:163BH         LINE#         752
  C:1646H         LINE#         753
  C:1651H         LINE#         754
  C:165CH         LINE#         755
  C:1665H         LINE#         758
  C:1670H         LINE#         759
  C:167BH         LINE#         760
  C:1686H         LINE#         761
  C:1691H         LINE#         762
  C:1698H         LINE#         764
  C:169BH         LINE#         765
  C:16A2H         LINE#         766
  C:16A7H         LINE#         767
  C:16AEH         LINE#         769
  C:16B7H         LINE#         770
  C:16C0H         LINE#         771
  C:16CAH         LINE#         772
  C:16CDH         LINE#         773
  C:16E4H         LINE#         774
  C:16ECH         LINE#         775
  C:16ECH         LINE#         776
  C:16F3H         LINE#         777
  C:16F3H         LINE#         778
  C:16F3H         LINE#         779
  C:16F6H         LINE#         780
  C:16F6H         LINE#         781
  C:1705H         LINE#         782
  C:1705H         LINE#         783
  C:170CH         LINE#         784
  C:1714H         LINE#         785
  C:171BH         LINE#         786
BL51 BANKED LINKER/LOCATER V4.13                                                      04/17/2013  16:59:47  PAGE 22


  C:1723H         LINE#         787
  C:172BH         LINE#         788
  C:1733H         LINE#         789
  C:173BH         LINE#         790
  C:1746H         LINE#         791
  C:174DH         LINE#         792
  C:1758H         LINE#         793
  C:1763H         LINE#         795
  C:176EH         LINE#         796
  C:1779H         LINE#         797
  C:1784H         LINE#         798
  C:178FH         LINE#         799
  C:179AH         LINE#         800
  C:17A5H         LINE#         801
  C:17B0H         LINE#         802
  C:17BBH         LINE#         803
  C:17C6H         LINE#         804
  C:17D1H         LINE#         808
  C:17DCH         LINE#         809
  C:17E7H         LINE#         810
  C:17F2H         LINE#         811
  C:17FDH         LINE#         812
  C:1808H         LINE#         813
  C:180FH         LINE#         814
  C:181AH         LINE#         815
  C:1825H         LINE#         816
  C:1830H         LINE#         818
  C:183BH         LINE#         819
  C:1844H         LINE#         821
  C:184FH         LINE#         822
  C:1858H         LINE#         823
  C:1861H         LINE#         824
  C:186AH         LINE#         825
  C:1875H         LINE#         826
  C:187CH         LINE#         827
  C:1887H         LINE#         828
  C:1890H         LINE#         829
  C:189BH         LINE#         830
  C:18A4H         LINE#         831
  C:18AFH         LINE#         832
  C:18B8H         LINE#         833
  C:18C1H         LINE#         834
  C:18CCH         LINE#         836
  C:18D7H         LINE#         837
  C:18DEH         LINE#         838
  C:18E1H         LINE#         839
  C:18F8H         LINE#         840
  C:1900H         LINE#         841
  C:1900H         LINE#         842
  C:1907H         LINE#         843
  C:1907H         LINE#         844
  C:1907H         LINE#         845
  C:190AH         LINE#         846
  C:190AH         LINE#         847
  C:1919H         LINE#         848
  C:1919H         LINE#         849
  C:1921H         LINE#         850
BL51 BANKED LINKER/LOCATER V4.13                                                      04/17/2013  16:59:47  PAGE 23


  C:1928H         LINE#         851
  C:1933H         LINE#         852
  C:193EH         LINE#         853
  C:1949H         LINE#         854
  C:1950H         LINE#         855
  C:195BH         LINE#         856
  C:1966H         LINE#         857
  C:196DH         LINE#         858
  C:1978H         LINE#         859
  C:197FH         LINE#         860
  C:198AH         LINE#         861
  C:1995H         LINE#         862
  C:199CH         LINE#         863
  C:19A7H         LINE#         864
  C:19B2H         LINE#         865
  C:19BDH         LINE#         866
  C:19C8H         LINE#         867
  C:19D3H         LINE#         868
  C:19DCH         LINE#         869
  C:19E7H         LINE#         870
  C:19F2H         LINE#         871
  C:19FDH         LINE#         872
  C:1A08H         LINE#         873
  C:1A13H         LINE#         874
  C:1A1EH         LINE#         875
  C:1A29H         LINE#         876
  C:1A34H         LINE#         877
  C:1A3FH         LINE#         878
  C:1A4AH         LINE#         879
  C:1A55H         LINE#         880
  C:1A60H         LINE#         881
  C:1A6BH         LINE#         882
  C:1A76H         LINE#         883
  C:1A81H         LINE#         884
  C:1A8CH         LINE#         885
  C:1A8FH         LINE#         886
  C:1A94H         LINE#         887
  C:1A99H         LINE#         888
  C:1A9EH         LINE#         889
  C:1AA5H         LINE#         890
  C:1AAEH         LINE#         891
  C:1AB1H         LINE#         892
  C:1AC8H         LINE#         893
  C:1AD0H         LINE#         894
  C:1AD0H         LINE#         895
  C:1AD7H         LINE#         896
  C:1AD7H         LINE#         897
  C:1AD7H         LINE#         898
  C:1ADAH         LINE#         899
  C:1ADAH         LINE#         900
  C:1AE9H         LINE#         901
  C:1AE9H         LINE#         902
  C:1AF2H         LINE#         903
  C:1AFDH         LINE#         904
  C:1B08H         LINE#         905
  C:1B13H         LINE#         906
  C:1B1EH         LINE#         907
BL51 BANKED LINKER/LOCATER V4.13                                                      04/17/2013  16:59:47  PAGE 24


  C:1B29H         LINE#         908
  C:1B30H         LINE#         909
  C:1B3BH         LINE#         910
  C:1B42H         LINE#         911
  C:1B4DH         LINE#         912
  C:1B58H         LINE#         913
  C:1B5FH         LINE#         914
  C:1B68H         LINE#         915
  C:1B73H         LINE#         916
  C:1B7EH         LINE#         917
  C:1B89H         LINE#         918
  C:1B94H         LINE#         919
  C:1B9FH         LINE#         920
  C:1BAAH         LINE#         921
  C:1BB5H         LINE#         922
  C:1BC0H         LINE#         923
  C:1BCBH         LINE#         925
  C:1BD6H         LINE#         926
  C:1BE1H         LINE#         927
  C:1BECH         LINE#         928
  C:1BF6H         LINE#         929
  C:1C01H         LINE#         930
  C:1C0CH         LINE#         931
  C:1C17H         LINE#         932
  C:1C22H         LINE#         933
  C:1C2DH         LINE#         934
  C:1C38H         LINE#         935
  C:1C43H         LINE#         936
  C:1C4EH         LINE#         937
  C:1C51H         LINE#         938
  C:1C56H         LINE#         939
  C:1C5BH         LINE#         940
  C:1C60H         LINE#         941
  C:1C67H         LINE#         942
  C:1C6AH         LINE#         943
  C:1C81H         LINE#         944
  C:1C89H         LINE#         945
  C:1C89H         LINE#         946
  C:1C90H         LINE#         947
  C:1C90H         LINE#         948
  C:1C90H         LINE#         949
  C:1C93H         LINE#         950
  C:1C93H         LINE#         951
  C:1C9EH         LINE#         952
  C:1C9EH         LINE#         953
  C:1CA0H         LINE#         954
  C:1CA6H         LINE#         955
  C:1CA8H         LINE#         956
  C:1CAFH         LINE#         957
  C:1CB1H         LINE#         958
  C:1CB3H         LINE#         959
  C:1CB5H         LINE#         960
  C:1CB7H         LINE#         961
  C:1CBEH         LINE#         964
  C:1CC9H         LINE#         965
  C:1CD4H         LINE#         966
  C:1CDDH         LINE#         967
BL51 BANKED LINKER/LOCATER V4.13                                                      04/17/2013  16:59:47  PAGE 25


  C:1CE8H         LINE#         968
  C:1CF3H         LINE#         969
  C:1CFEH         LINE#         970
  C:1D09H         LINE#         971
  C:1D14H         LINE#         972
  C:1D1FH         LINE#         973
  C:1D2AH         LINE#         974
  C:1D35H         LINE#         975
  C:1D40H         LINE#         978
  C:1D49H         LINE#         979
  C:1D52H         LINE#         980
  C:1D5BH         LINE#         981
  C:1D66H         LINE#         982
  C:1D6FH         LINE#         983
  C:1D78H         LINE#         984
  C:1D83H         LINE#         985
  C:1D8EH         LINE#         988
  C:1D99H         LINE#         989
  C:1DA4H         LINE#         990
  C:1DAFH         LINE#         991
  C:1DBAH         LINE#         992
  C:1DC5H         LINE#         994
  C:1DD0H         LINE#         995
  C:1DDBH         LINE#         996
  C:1DE6H         LINE#         997
  C:1DF1H         LINE#         998
  C:1DFCH         LINE#         999
  C:1E07H         LINE#         1001
  C:1E12H         LINE#         1002
  C:1E1BH         LINE#         1003
  C:1E26H         LINE#         1004
  C:1E2FH         LINE#         1005
  C:1E36H         LINE#         1006
  C:1E41H         LINE#         1007
  C:1E4CH         LINE#         1008
  C:1E57H         LINE#         1009
  C:1E62H         LINE#         1010
  C:1E6DH         LINE#         1013
  C:1E78H         LINE#         1014
  C:1E83H         LINE#         1015
  C:1E8AH         LINE#         1016
  C:1E95H         LINE#         1017
  C:1EA0H         LINE#         1018
  C:1EA9H         LINE#         1019
  C:1EB4H         LINE#         1022
  C:1EBFH         LINE#         1023
  C:1ECAH         LINE#         1024
  C:1ED1H         LINE#         1025
  C:1EDCH         LINE#         1026
  C:1EE3H         LINE#         1028
  C:1EEEH         LINE#         1029
  C:1EF5H         LINE#         1030
  C:1F00H         LINE#         1031
  C:1F07H         LINE#         1032
  C:1F12H         LINE#         1033
  C:1F19H         LINE#         1036
  C:1F24H         LINE#         1037
BL51 BANKED LINKER/LOCATER V4.13                                                      04/17/2013  16:59:47  PAGE 26


  C:1F2FH         LINE#         1038
  C:1F36H         LINE#         1039
  C:1F41H         LINE#         1040
  C:1F4CH         LINE#         1041
  C:1F53H         LINE#         1042
  C:1F5EH         LINE#         1045
  C:1F69H         LINE#         1046
  C:1F74H         LINE#         1047
  C:1F7DH         LINE#         1049
  C:1F84H         LINE#         1050
  C:1F87H         LINE#         1051
  C:1F9EH         LINE#         1052
  C:1FA6H         LINE#         1053
  C:1FA6H         LINE#         1054
  C:1FADH         LINE#         1055
  C:1FADH         LINE#         1056
  C:1FADH         LINE#         1057
  C:1FB0H         LINE#         1058
  C:1FB0H         LINE#         1059
  C:1FBBH         LINE#         1060
  C:1FBBH         LINE#         1061
  C:1FBDH         LINE#         1062
  C:1FC3H         LINE#         1063
  C:1FC5H         LINE#         1064
  C:1FCCH         LINE#         1065
  C:1FCEH         LINE#         1066
  C:1FD0H         LINE#         1067
  C:1FD2H         LINE#         1068
  C:1FD4H         LINE#         1069
  C:1FDBH         LINE#         1072
  C:1FE6H         LINE#         1073
  C:1FF1H         LINE#         1074
  C:1FFAH         LINE#         1075
  C:2005H         LINE#         1076
  C:2010H         LINE#         1077
  C:201BH         LINE#         1078
  C:2026H         LINE#         1079
  C:2031H         LINE#         1080
  C:203CH         LINE#         1081
  C:2047H         LINE#         1082
  C:2052H         LINE#         1083
  C:205DH         LINE#         1086
  C:2066H         LINE#         1087
  C:206FH         LINE#         1088
  C:2078H         LINE#         1089
  C:2083H         LINE#         1090
  C:208CH         LINE#         1091
  C:2095H         LINE#         1092
  C:20A0H         LINE#         1093
  C:20ABH         LINE#         1096
  C:20B6H         LINE#         1097
  C:20C1H         LINE#         1098
  C:20CCH         LINE#         1099
  C:20D7H         LINE#         1100
  C:20E2H         LINE#         1102
  C:20EDH         LINE#         1103
  C:20F8H         LINE#         1104
BL51 BANKED LINKER/LOCATER V4.13                                                      04/17/2013  16:59:47  PAGE 27


  C:2103H         LINE#         1105
  C:210EH         LINE#         1106
  C:2119H         LINE#         1107
  C:2124H         LINE#         1109
  C:212FH         LINE#         1110
  C:2138H         LINE#         1111
  C:2143H         LINE#         1112
  C:214CH         LINE#         1113
  C:2153H         LINE#         1114
  C:215EH         LINE#         1115
  C:2169H         LINE#         1116
  C:2174H         LINE#         1117
  C:217FH         LINE#         1118
  C:218AH         LINE#         1121
  C:2195H         LINE#         1122
  C:21A0H         LINE#         1123
  C:21A7H         LINE#         1124
  C:21B2H         LINE#         1125
  C:21BDH         LINE#         1126
  C:21C6H         LINE#         1127
  C:21D1H         LINE#         1130
  C:21DCH         LINE#         1131
  C:21E7H         LINE#         1132
  C:21EEH         LINE#         1133
  C:21F9H         LINE#         1134
  C:2200H         LINE#         1136
  C:220BH         LINE#         1137
  C:2212H         LINE#         1138
  C:221DH         LINE#         1139
  C:2224H         LINE#         1140
  C:222FH         LINE#         1141
  C:2236H         LINE#         1144
  C:2241H         LINE#         1145
  C:224CH         LINE#         1146
  C:2253H         LINE#         1147
  C:225EH         LINE#         1148
  C:2269H         LINE#         1149
  C:2270H         LINE#         1150
  C:227BH         LINE#         1153
  C:2286H         LINE#         1154
  C:2291H         LINE#         1155
  C:229AH         LINE#         1157
  C:22A1H         LINE#         1158
  C:22A1H         LINE#         1160
  -------         ENDPROC       LCD_INIT
  -------         PROC          _LCD_ID
  D:0010H         SYMBOL        dat
  -------         DO            dat
  D:0012H         SYMBOL        temp
  D:0014H         SYMBOL        DH
  D:0016H         SYMBOL        DL
  D:0012H         SYMBOL        temp
  D:0014H         SYMBOL        DH
  D:0016H         SYMBOL        DL
  -------         ENDDO         DL
  -------         DO            DL
  D:0012H         SYMBOL        temp
BL51 BANKED LINKER/LOCATER V4.13                                                      04/17/2013  16:59:47  PAGE 28


  D:0014H         SYMBOL        DH
  D:0016H         SYMBOL        DL
  -------         ENDDO         DL
  C:30EDH         LINE#         1166
  C:30F1H         LINE#         1167
  C:30F1H         LINE#         1168
  C:30F9H         LINE#         1169
  C:30F9H         LINE#         1171
  C:30FDH         LINE#         1172
  C:3100H         LINE#         1173
  C:3105H         LINE#         1174
  C:3108H         LINE#         1175
  C:310BH         LINE#         1177
  C:310DH         LINE#         1178
  C:310FH         LINE#         1179
  C:3111H         LINE#         1180
  C:3117H         LINE#         1181
  C:311EH         LINE#         1183
  C:3120H         LINE#         1184
  C:3122H         LINE#         1185
  C:3129H         LINE#         1189
  C:312BH         LINE#         1190
  C:312DH         LINE#         1191
  C:3133H         LINE#         1193
  C:313BH         LINE#         1194
  C:3142H         LINE#         1195
  C:314AH         LINE#         1197
  C:314FH         LINE#         1198
  C:314FH         LINE#         1199
  C:314FH         LINE#         1201
  C:3156H         LINE#         1202
  C:315BH         LINE#         1203
  C:315EH         LINE#         1204
  C:3161H         LINE#         1206
  C:3163H         LINE#         1207
  C:3165H         LINE#         1208
  C:3167H         LINE#         1209
  C:316DH         LINE#         1211
  C:3174H         LINE#         1212
  C:317BH         LINE#         1215
  C:317DH         LINE#         1219
  C:317FH         LINE#         1221
  C:3187H         LINE#         1222
  C:318EH         LINE#         1223
  C:3196H         LINE#         1225
  C:319AH         LINE#         1226
  C:319AH         LINE#         1227
  -------         ENDPROC       _LCD_ID
  -------         PROC          _LCD_ID_61581
  D:0010H         SYMBOL        dat
  -------         DO            dat
  D:0012H         SYMBOL        temp
  D:0014H         SYMBOL        DH
  D:0016H         SYMBOL        DL
  -------         ENDDO         DL
  C:319BH         LINE#         1232
  C:319FH         LINE#         1233
BL51 BANKED LINKER/LOCATER V4.13                                                      04/17/2013  16:59:47  PAGE 29


  C:319FH         LINE#         1237
  C:31A6H         LINE#         1238
  C:31ACH         LINE#         1240
  C:31B3H         LINE#         1241
  C:31B8H         LINE#         1242
  C:31BBH         LINE#         1243
  C:31BEH         LINE#         1245
  C:31C0H         LINE#         1246
  C:31C2H         LINE#         1247
  C:31C4H         LINE#         1248
  C:31CAH         LINE#         1250
  C:31CAH         LINE#         1251
  C:31CAH         LINE#         1253
  C:31CAH         LINE#         1254
  C:31CAH         LINE#         1255
  C:31CAH         LINE#         1257
  C:31CAH         LINE#         1258
  C:31CAH         LINE#         1259
  C:31CAH         LINE#         1260
  C:31CDH         LINE#         1262
  C:31CDH         LINE#         1263
  C:31CDH         LINE#         1265
  C:31CDH         LINE#         1266
  C:31CDH         LINE#         1267
  C:31CDH         LINE#         1269
  C:31CDH         LINE#         1270
  C:31CDH         LINE#         1271
  C:31CDH         LINE#         1272
  C:31D0H         LINE#         1274
  C:31D0H         LINE#         1275
  C:31D0H         LINE#         1277
  C:31D0H         LINE#         1278
  C:31D0H         LINE#         1279
  C:31D0H         LINE#         1283
  C:31D0H         LINE#         1284
  C:31D0H         LINE#         1285
  C:31D0H         LINE#         1286
  C:31D3H         LINE#         1288
  C:31DAH         LINE#         1289
  C:31E1H         LINE#         1291
  C:31E3H         LINE#         1292
  C:31E8H         LINE#         1293
  C:31EDH         LINE#         1295
  C:31F5H         LINE#         1296
  C:31FCH         LINE#         1298
  C:31FCH         LINE#         1299
  C:31FCH         LINE#         1300
  C:31FCH         LINE#         1301
  C:31FFH         LINE#         1303
  C:3206H         LINE#         1304
  C:320DH         LINE#         1306
  C:320FH         LINE#         1307
  C:3214H         LINE#         1308
  C:3219H         LINE#         1312
  C:321BH         LINE#         1316
  C:3223H         LINE#         1318
  C:3227H         LINE#         1319
BL51 BANKED LINKER/LOCATER V4.13                                                      04/17/2013  16:59:47  PAGE 30


  -------         ENDPROC       _LCD_ID_61581
  -------         PROC          LCD_READ_ID61581
  -------         DO            LCD_READ_ID61581
  D:0005H         SYMBOL        m
  D:0004H         SYMBOL        n
  -------         ENDDO         n
  C:3682H         LINE#         1324
  C:3682H         LINE#         1325
  C:3682H         LINE#         1328
  C:3682H         LINE#         1329
  C:3682H         LINE#         1330
  C:3685H         LINE#         1331
  C:368CH         LINE#         1333
  C:3697H         LINE#         1336
  C:3699H         LINE#         1337
  C:3699H         LINE#         1338
  C:3699H         LINE#         1340
  C:3699H         LINE#         1341
  C:3699H         LINE#         1342
  C:3699H         LINE#         1344
  C:3699H         LINE#         1345
  -------         ENDPROC       LCD_READ_ID61581
  -------         PROC          _LCD_ID_9341
  D:0004H         SYMBOL        dat
  -------         DO            dat
  D:0010H         SYMBOL        temp
  D:0012H         SYMBOL        DH
  D:0014H         SYMBOL        DL
  -------         ENDDO         DL
  C:3036H         LINE#         1352
  C:303AH         LINE#         1353
  C:303AH         LINE#         1354
  C:3042H         LINE#         1355
  C:3042H         LINE#         1356
  C:3046H         LINE#         1357
  C:3046H         LINE#         1358
  C:3046H         LINE#         1360
  C:304DH         LINE#         1361
  C:3052H         LINE#         1362
  C:3055H         LINE#         1363
  C:3058H         LINE#         1365
  C:305AH         LINE#         1366
  C:305CH         LINE#         1367
  C:305EH         LINE#         1368
  C:3064H         LINE#         1370
  C:306BH         LINE#         1371
  C:3072H         LINE#         1373
  C:3074H         LINE#         1374
  C:3079H         LINE#         1375
  C:307BH         LINE#         1377
  C:307BH         LINE#         1378
  C:307BH         LINE#         1379
  C:307BH         LINE#         1380
  C:307EH         LINE#         1382
  C:3085H         LINE#         1383
  C:308CH         LINE#         1385
  C:308EH         LINE#         1386
BL51 BANKED LINKER/LOCATER V4.13                                                      04/17/2013  16:59:47  PAGE 31


  C:3093H         LINE#         1387
  C:3095H         LINE#         1389
  C:3095H         LINE#         1390
  C:3095H         LINE#         1391
  C:3095H         LINE#         1392
  C:3098H         LINE#         1394
  C:309FH         LINE#         1395
  C:30A6H         LINE#         1397
  C:30A8H         LINE#         1398
  C:30ADH         LINE#         1399
  C:30B2H         LINE#         1401
  C:30BAH         LINE#         1402
  C:30C1H         LINE#         1407
  C:30C1H         LINE#         1408
  C:30C1H         LINE#         1409
  C:30C1H         LINE#         1410
  C:30C4H         LINE#         1412
  C:30CBH         LINE#         1413
  C:30D2H         LINE#         1415
  C:30D4H         LINE#         1416
  C:30D9H         LINE#         1417
  C:30DEH         LINE#         1421
  C:30E0H         LINE#         1424
  C:30E8H         LINE#         1426
  C:30ECH         LINE#         1427
  C:30ECH         LINE#         1428
  -------         ENDPROC       _LCD_ID_9341
  -------         PROC          LCD_READ_8347ID
  -------         DO            LCD_READ_8347ID
  D:0005H         SYMBOL        m
  D:0004H         SYMBOL        n
  -------         ENDDO         n
  C:3618H         LINE#         1433
  C:3618H         LINE#         1434
  C:3618H         LINE#         1437
  C:3618H         LINE#         1438
  C:361BH         LINE#         1439
  C:3622H         LINE#         1440
  C:362CH         LINE#         1441
  C:3633H         LINE#         1442
  C:363AH         LINE#         1443
  C:363AH         LINE#         1445
  C:363AH         LINE#         1446
  C:363AH         LINE#         1447
  C:363AH         LINE#         1449
  C:363AH         LINE#         1450
  C:363AH         LINE#         1451
  C:363AH         LINE#         1453
  C:363AH         LINE#         1454
  -------         ENDPROC       LCD_READ_8347ID
  -------         PROC          LCD_READ_ID
  -------         DO            LCD_READ_ID
  D:0005H         SYMBOL        m
  D:0004H         SYMBOL        n
  -------         ENDDO         n
  C:363DH         LINE#         1460
  C:363DH         LINE#         1461
BL51 BANKED LINKER/LOCATER V4.13                                                      04/17/2013  16:59:47  PAGE 32


  C:363DH         LINE#         1464
  C:363DH         LINE#         1465
  C:3640H         LINE#         1466
  C:3647H         LINE#         1467
  C:3651H         LINE#         1468
  C:3658H         LINE#         1469
  C:365EH         LINE#         1470
  C:365EH         LINE#         1472
  C:365EH         LINE#         1473
  C:365EH         LINE#         1474
  C:365EH         LINE#         1476
  C:365EH         LINE#         1477
  C:365EH         LINE#         1478
  C:365EH         LINE#         1480
  C:365EH         LINE#         1481
  -------         ENDPROC       LCD_READ_ID
  -------         PROC          LCD_READ_ID9341
  -------         DO            LCD_READ_ID9341
  D:0005H         SYMBOL        m
  D:0004H         SYMBOL        n
  -------         ENDDO         n
  C:3661H         LINE#         1487
  C:3661H         LINE#         1488
  C:3661H         LINE#         1491
  C:3661H         LINE#         1492
  C:3661H         LINE#         1493
  C:3664H         LINE#         1494
  C:366BH         LINE#         1495
  C:3672H         LINE#         1496
  C:367DH         LINE#         1499
  C:367FH         LINE#         1500
  C:367FH         LINE#         1501
  C:367FH         LINE#         1503
  C:367FH         LINE#         1504
  C:367FH         LINE#         1505
  C:367FH         LINE#         1507
  C:367FH         LINE#         1508
  -------         ENDPROC       LCD_READ_ID9341
  C:369FH         SYMBOL        L?0196
  -------         PROC          L?0195
  -------         ENDPROC       L?0195
  C:369FH         SYMBOL        L?0196
  -------         PROC          HD_RESET
  C:36A4H         LINE#         1515
  C:36A4H         LINE#         1516
  C:36A4H         LINE#         1517
  C:36A6H         LINE#         1518
  C:36ADH         LINE#         1519
  C:36AFH         LINE#         1520
  -------         ENDPROC       HD_RESET
  -------         PROC          _LCD_WRITE_CMD
  D:0007H         SYMBOL        cmd1
  D:0005H         SYMBOL        cmd2
  C:3590H         LINE#         1526
  C:3590H         LINE#         1527
  C:3590H         LINE#         1528
  C:3598H         LINE#         1529
BL51 BANKED LINKER/LOCATER V4.13                                                      04/17/2013  16:59:47  PAGE 33


  C:3598H         LINE#         1530
  C:359AH         LINE#         1531
  C:359CH         LINE#         1532
  C:359EH         LINE#         1533
  C:35A0H         LINE#         1534
  C:35A2H         LINE#         1535
  C:35A4H         LINE#         1537
  C:35A6H         LINE#         1538
  C:35A8H         LINE#         1539
  C:35AAH         LINE#         1541
  C:35ACH         LINE#         1542
  C:35AEH         LINE#         1543
  C:35AFH         LINE#         1544
  C:35AFH         LINE#         1545
  C:35B1H         LINE#         1546
  C:35B3H         LINE#         1547
  C:35B5H         LINE#         1548
  C:35B7H         LINE#         1549
  C:35B9H         LINE#         1551
  C:35BBH         LINE#         1552
  C:35BDH         LINE#         1554
  C:35BFH         LINE#         1555
  C:35C1H         LINE#         1556
  C:35C1H         LINE#         1557
  -------         ENDPROC       _LCD_WRITE_CMD
  C:335EH         SYMBOL        L?0187
  C:335FH         SYMBOL        L?0188
  -------         PROC          L?0186
  -------         ENDPROC       L?0186
  C:335EH         SYMBOL        L?0187
  C:335FH         SYMBOL        L?0188
  -------         PROC          _LCD_WRITE_DATA
  D:0007H         SYMBOL        dataa
  D:0005H         SYMBOL        datab
  C:3364H         LINE#         1562
  C:3364H         LINE#         1563
  C:3364H         LINE#         1564
  C:336CH         LINE#         1565
  C:336CH         LINE#         1566
  C:336EH         LINE#         1567
  C:3370H         LINE#         1568
  C:3372H         LINE#         1569
  C:3374H         LINE#         1570
  C:3376H         LINE#         1571
  C:3378H         LINE#         1573
  C:337AH         LINE#         1574
  C:337CH         LINE#         1575
  C:337EH         LINE#         1577
  C:3380H         LINE#         1578
  C:3382H         LINE#         1579
  C:3383H         LINE#         1580
  C:3383H         LINE#         1581
  C:3385H         LINE#         1582
  C:3387H         LINE#         1583
  C:3389H         LINE#         1584
  C:338BH         LINE#         1585
  C:338DH         LINE#         1587
BL51 BANKED LINKER/LOCATER V4.13                                                      04/17/2013  16:59:47  PAGE 34


  C:338FH         LINE#         1588
  C:3391H         LINE#         1590
  C:3393H         LINE#         1591
  C:3395H         LINE#         1592
  C:3395H         LINE#         1593
  -------         ENDPROC       _LCD_WRITE_DATA
  -------         PROC          L?0194
  -------         ENDPROC       L?0194
  -------         PROC          _LLCD_WRITE_CMD
  D:0004H         SYMBOL        cmd
  C:33B8H         LINE#         1598
  C:33BCH         LINE#         1599
  C:33BCH         LINE#         1600
  C:33C4H         LINE#         1601
  C:33C4H         LINE#         1602
  C:33C6H         LINE#         1603
  C:33C8H         LINE#         1604
  C:33CAH         LINE#         1605
  C:33CCH         LINE#         1606
  C:33D3H         LINE#         1607
  C:33D5H         LINE#         1609
  C:33D7H         LINE#         1610
  C:33D9H         LINE#         1611
  C:33DBH         LINE#         1613
  C:33DDH         LINE#         1614
  C:33DFH         LINE#         1615
  C:33E0H         LINE#         1616
  C:33E0H         LINE#         1617
  C:33E2H         LINE#         1618
  C:33E4H         LINE#         1619
  C:33E6H         LINE#         1620
  C:33E8H         LINE#         1621
  C:33EFH         LINE#         1623
  C:33F1H         LINE#         1624
  C:33F3H         LINE#         1626
  C:33F5H         LINE#         1627
  C:33F7H         LINE#         1628
  C:33F7H         LINE#         1629
  -------         ENDPROC       _LLCD_WRITE_CMD
  -------         PROC          L?0193
  -------         ENDPROC       L?0193
  -------         PROC          _LLCD_WRITE_DATA
  D:0004H         SYMBOL        dataa
  C:3494H         LINE#         1634
  C:3498H         LINE#         1635
  C:3498H         LINE#         1636
  C:34A0H         LINE#         1637
  C:34A0H         LINE#         1638
  C:34A2H         LINE#         1639
  C:34A4H         LINE#         1640
  C:34A6H         LINE#         1641
  C:34A8H         LINE#         1642
  C:34AFH         LINE#         1643
  C:34B1H         LINE#         1645
  C:34B3H         LINE#         1646
  C:34B5H         LINE#         1647
  C:34B7H         LINE#         1649
BL51 BANKED LINKER/LOCATER V4.13                                                      04/17/2013  16:59:47  PAGE 35


  C:34B9H         LINE#         1650
  C:34BBH         LINE#         1651
  C:34BCH         LINE#         1652
  C:34BCH         LINE#         1653
  C:34BEH         LINE#         1654
  C:34C0H         LINE#         1655
  C:34C2H         LINE#         1656
  C:34C4H         LINE#         1657
  C:34CBH         LINE#         1662
  C:34CDH         LINE#         1663
  C:34CFH         LINE#         1665
  C:34D1H         LINE#         1666
  C:34D3H         LINE#         1667
  C:34D3H         LINE#         1668
  -------         ENDPROC       _LLCD_WRITE_DATA
  C:36CFH         SYMBOL        L?0183
  C:36D1H         SYMBOL        L?0184
  C:36D3H         SYMBOL        L?0185
  -------         PROC          L?0182
  -------         ENDPROC       L?0182
  C:36CFH         SYMBOL        L?0183
  C:36D1H         SYMBOL        L?0184
  C:36D3H         SYMBOL        L?0185
  -------         PROC          _SENG_CMD_DAT
  D:0006H         SYMBOL        cmd
  D:0002H         SYMBOL        dataa
  C:36D7H         LINE#         1674
  C:36DBH         LINE#         1675
  C:36DBH         LINE#         1676
  C:36DEH         LINE#         1677
  -------         ENDPROC       _SENG_CMD_DAT
  C:33F8H         SYMBOL        L?0175
  C:33FDH         SYMBOL        L?0176
  -------         PROC          L?0174
  -------         ENDPROC       L?0174
  C:33F8H         SYMBOL        L?0175
  C:33FDH         SYMBOL        L?0176
  -------         PROC          _GUI_SPRINTF_STRING
  D:0010H         SYMBOL        x
  D:0011H         SYMBOL        y
  D:0013H         SYMBOL        s
  D:0015H         SYMBOL        color
  D:0017H         SYMBOL        b_color
  C:340CH         LINE#         1683
  C:3416H         LINE#         1684
  C:3416H         LINE#         1685
  C:3421H         LINE#         1686
  C:3421H         LINE#         1687
  C:3436H         LINE#         1688
  C:343CH         LINE#         1689
  C:3446H         LINE#         1692
  -------         ENDPROC       _GUI_SPRINTF_STRING
  -------         PROC          _GUI_SPRINTF_CHAR
  D:0019H         SYMBOL        x
  D:001AH         SYMBOL        y
  D:001CH         SYMBOL        c
  D:001DH         SYMBOL        color
BL51 BANKED LINKER/LOCATER V4.13                                                      04/17/2013  16:59:47  PAGE 36


  D:001FH         SYMBOL        b_color
  -------         DO            b_color
  D:0021H         SYMBOL        s_x
  D:0022H         SYMBOL        s_y
  D:0023H         SYMBOL        temp
  D:0002H         SYMBOL        j
  -------         ENDDO         j
  C:2F6DH         LINE#         1697
  C:2F75H         LINE#         1698
  C:2F75H         LINE#         1701
  C:2F7BH         LINE#         1702
  C:2F7EH         LINE#         1703
  C:2F7EH         LINE#         1704
  C:2F96H         LINE#         1705
  C:2F96H         LINE#         1706
  C:2F9AH         LINE#         1707
  C:2FAEH         LINE#         1708
  C:2FBDH         LINE#         1710
  C:2FC0H         LINE#         1711
  C:2FC0H         LINE#         1712
  C:2FD3H         LINE#         1713
  C:2FD3H         LINE#         1714
  C:2FF2H         LINE#         1715
  C:2FF2H         LINE#         1716
  C:3007H         LINE#         1717
  C:3009H         LINE#         1719
  C:3009H         LINE#         1720
  C:3020H         LINE#         1721
  C:3020H         LINE#         1722
  C:3020H         LINE#         1723
  C:3029H         LINE#         1724
  C:3029H         LINE#         1725
  C:3035H         LINE#         1726
  -------         ENDPROC       _GUI_SPRINTF_CHAR
  -------         PROC          _GUI_POINT
  D:0007H         SYMBOL        x
  D:0004H         SYMBOL        y
  D:0024H         SYMBOL        color
  C:36F4H         LINE#         1731
  C:36F8H         LINE#         1732
  C:36F8H         LINE#         1733
  C:36FBH         LINE#         1734
  -------         ENDPROC       _GUI_POINT
  -------         PROC          _LCD_SETXY
  D:0003H         SYMBOL        x
  D:0004H         SYMBOL        y
  C:3732H         LINE#         1740
  C:3734H         LINE#         1741
  C:3734H         LINE#         1742
  -------         ENDPROC       _LCD_SETXY
  -------         PROC          _LCD_SETWINDOW
  D:0001H         SYMBOL        x0
  D:0027H         SYMBOL        y0
  D:0029H         SYMBOL        x1
  D:002AH         SYMBOL        y1
  C:2E74H         LINE#         1748
  C:2E7CH         LINE#         1749
BL51 BANKED LINKER/LOCATER V4.13                                                      04/17/2013  16:59:47  PAGE 37


  C:2E7CH         LINE#         1750
  C:2E87H         LINE#         1751
  C:2E93H         LINE#         1752
  C:2E9EH         LINE#         1753
  C:2EA9H         LINE#         1754
  C:2EB3H         LINE#         1755
  C:2EB3H         LINE#         1756
  C:2EBEH         LINE#         1757
  C:2EC9H         LINE#         1758
  C:2ED0H         LINE#         1759
  C:2EDCH         LINE#         1760
  C:2EDCH         LINE#         1761
  C:2EDCH         LINE#         1762
  C:2EDCH         LINE#         1763
  C:2EDCH         LINE#         1765
  C:2EDCH         LINE#         1766
  C:2EDCH         LINE#         1767
  C:2EDCH         LINE#         1769
  C:2EDFH         LINE#         1770
  C:2EEBH         LINE#         1771
  C:2EEBH         LINE#         1772
  C:2EEBH         LINE#         1773
  C:2EEBH         LINE#         1774
  C:2EEBH         LINE#         1776
  C:2EEBH         LINE#         1777
  C:2EEBH         LINE#         1778
  C:2EEBH         LINE#         1780
  C:2EEEH         LINE#         1781
  C:2EEEH         LINE#         1782
  C:2EF6H         LINE#         1783
  C:2EF6H         LINE#         1784
  C:2EFEH         LINE#         1785
  C:2F09H         LINE#         1786
  C:2F12H         LINE#         1787
  C:2F1EH         LINE#         1788
  C:2F2AH         LINE#         1789
  C:2F31H         LINE#         1790
  C:2F3DH         LINE#         1791
  C:2F48H         LINE#         1792
  C:2F4FH         LINE#         1793
  C:2F4FH         LINE#         1795
  C:2F4FH         LINE#         1796
  C:2F5AH         LINE#         1797
  C:2F65H         LINE#         1798
  C:2F6CH         LINE#         1799
  C:2F6CH         LINE#         1801
  -------         ENDPROC       _LCD_SETWINDOW
  C:2C27H         SYMBOL        L?0192
  -------         PROC          L?0191
  -------         ENDPROC       L?0191
  C:2C27H         SYMBOL        L?0192
  -------         PROC          _LCD_TEST_SINGLECOLOR
  D:0010H         SYMBOL        colorH
  D:0001H         SYMBOL        colorL
  -------         DO            colorL
  D:0011H         SYMBOL        i
  D:0002H         SYMBOL        j
BL51 BANKED LINKER/LOCATER V4.13                                                      04/17/2013  16:59:47  PAGE 38


  -------         ENDDO         j
  C:2C2BH         LINE#         1806
  C:2C2FH         LINE#         1807
  C:2C2FH         LINE#         1809
  C:2C3BH         LINE#         1810
  C:2C3BH         LINE#         1811
  C:2C41H         LINE#         1812
  C:2C4DH         LINE#         1813
  C:2C52H         LINE#         1814
  C:2C5EH         LINE#         1816
  C:2C64H         LINE#         1817
  C:2C69H         LINE#         1818
  C:2C6EH         LINE#         1819
  C:2C73H         LINE#         1822
  C:2C7AH         LINE#         1823
  C:2C7FH         LINE#         1824
  C:2C85H         LINE#         1825
  C:2C94H         LINE#         1826
  C:2C94H         LINE#         1827
  C:2C94H         LINE#         1828
  C:2C94H         LINE#         1829
  C:2C94H         LINE#         1830
  C:2C94H         LINE#         1834
  C:2C94H         LINE#         1835
  C:2C97H         LINE#         1836
  C:2C9DH         LINE#         1837
  C:2CACH         LINE#         1838
  C:2CACH         LINE#         1839
  C:2CACH         LINE#         1840
  C:2CACH         LINE#         1841
  C:2CACH         LINE#         1842
  C:2CACH         LINE#         1846
  C:2CACH         LINE#         1847
  C:2CAFH         LINE#         1848
  C:2CB5H         LINE#         1849
  C:2CB7H         LINE#         1852
  C:2CB7H         LINE#         1853
  C:2CBEH         LINE#         1854
  C:2CCAH         LINE#         1855
  C:2CCFH         LINE#         1856
  C:2CDBH         LINE#         1860
  C:2CE2H         LINE#         1861
  C:2CE7H         LINE#         1862
  C:2CEDH         LINE#         1863
  C:2CEDH         LINE#         1864
  C:2CF7H         LINE#         1865
  C:2CF7H         LINE#         1866
  C:2CFCH         LINE#         1867
  C:2CFCH         LINE#         1868
  C:2CFFH         LINE#         1869
  C:2CFFH         LINE#         1870
  C:2D06H         LINE#         1871
  C:2D11H         LINE#         1872
  C:2D25H         LINE#         1873
  C:2D25H         LINE#         1874
  C:2D25H         LINE#         1875
  C:2D2AH         LINE#         1876
BL51 BANKED LINKER/LOCATER V4.13                                                      04/17/2013  16:59:47  PAGE 39


  C:2D2AH         LINE#         1877
  C:2D2DH         LINE#         1878
  C:2D2DH         LINE#         1879
  C:2D34H         LINE#         1880
  C:2D3FH         LINE#         1881
  C:2D52H         LINE#         1882
  C:2D52H         LINE#         1883
  -------         ENDPROC       _LCD_TEST_SINGLECOLOR
  -------         PROC          KEYPRESS
  C:3702H         LINE#         1888
  C:3702H         LINE#         1889
  C:3702H         LINE#         1890
  C:3705H         LINE#         1891
  C:370EH         LINE#         1892
  -------         ENDPROC       KEYPRESS
  C:3515H         SYMBOL        L?0178
  C:352CH         SYMBOL        L?0179
  C:352FH         SYMBOL        L?0180
  C:3535H         SYMBOL        L?0181
  -------         PROC          L?0177
  -------         ENDPROC       L?0177
  C:3515H         SYMBOL        L?0178
  C:352CH         SYMBOL        L?0179
  C:352FH         SYMBOL        L?0180
  C:3535H         SYMBOL        L?0181
  -------         PROC          _DELAYMS
  D:0018H         SYMBOL        value
  C:3539H         LINE#         1897
  C:353DH         LINE#         1898
  C:353DH         LINE#         1899
  C:3543H         LINE#         1900
  C:3543H         LINE#         1901
  C:354AH         LINE#         1902
  C:3552H         LINE#         1903
  C:3554H         LINE#         1904
  -------         ENDPROC       _DELAYMS
  -------         PROC          _DELAYUS
  D:0006H         SYMBOL        value1
  C:370FH         LINE#         1909
  C:370FH         LINE#         1910
  C:370FH         LINE#         1911
  C:3713H         LINE#         1912
  C:371AH         LINE#         1913
  -------         ENDPROC       _DELAYUS
  -------         ENDMOD        LCD_DRIVE

  -------         MODULE        TOUCH
  C:0000H         SYMBOL        _ICE_DUMMY_
  C:373BH         PUBLIC        spistart
  D:0090H         PUBLIC        P1
  D:00B0H         PUBLIC        P3
  B:00B0H.4       PUBLIC        T0
  B:00D0H.6       PUBLIC        AC
  C:35F2H         PUBLIC        ReadFromCharFrom7843
  B:00B0H.5       PUBLIC        T1
  B:0090H.0       PUBLIC        T2
  B:00A8H.7       PUBLIC        EA
BL51 BANKED LINKER/LOCATER V4.13                                                      04/17/2013  16:59:47  PAGE 40


  C:36B6H         PUBLIC        _WriteCharTo7843
  D:00A8H         PUBLIC        IE
  B:00B0H.7       PUBLIC        CS
  B:00C8H.6       PUBLIC        EXF2
  B:00B0H.7       PUBLIC        RD
  B:00A8H.4       PUBLIC        ES
  D:00B8H         PUBLIC        IP
  B:0098H.0       PUBLIC        RI
  B:00B0H.2       PUBLIC        INT0
  B:00D0H.7       PUBLIC        CY
  B:0098H.1       PUBLIC        TI
  B:00B0H.3       PUBLIC        INT1
  B:00B0H.6       PUBLIC        DCLK
  B:00B8H.4       PUBLIC        PS
  B:0090H.1       PUBLIC        T2EX
  B:0090H.1       PUBLIC        RS
  B:00D0H.2       PUBLIC        OV
  B:00C8H.1       PUBLIC        C_T2
  B:00B0H.6       PUBLIC        WR
  B:00C8H.5       PUBLIC        RCLK
  B:00C8H.4       PUBLIC        TCLK
  D:0098H         PUBLIC        SCON
  D:0088H         PUBLIC        TCON
  B:00B0H.4       PUBLIC        DOUT
  C:32ABH         PUBLIC        INRT
  C:34D4H         PUBLIC        _drawpoint
  B:0088H.1       PUBLIC        IE0
  B:0088H.3       PUBLIC        IE1
  B:00B0H.3       PUBLIC        BUSY
  B:00C8H.0       PUBLIC        CP_RL2
  B:00A8H.1       PUBLIC        ET0
  B:00A8H.3       PUBLIC        ET1
  B:0088H.5       PUBLIC        TF0
  B:00A8H.5       PUBLIC        ET2
  B:0088H.7       PUBLIC        TF1
  B:00C8H.7       PUBLIC        TF2
  B:0098H.2       PUBLIC        RB8
  B:00A8H.0       PUBLIC        EX0
  B:0088H.0       PUBLIC        IT0
  B:0098H.3       PUBLIC        TB8
  B:00A8H.2       PUBLIC        EX1
  B:0088H.2       PUBLIC        IT1
  B:00D0H.0       PUBLIC        P
  B:0098H.7       PUBLIC        SM0
  B:0098H.6       PUBLIC        SM1
  B:0098H.5       PUBLIC        SM2
  B:00B8H.1       PUBLIC        PT0
  B:00B8H.3       PUBLIC        PT1
  B:00D0H.3       PUBLIC        RS0
  B:00B8H.5       PUBLIC        PT2
  B:0088H.4       PUBLIC        TR0
  B:00D0H.4       PUBLIC        RS1
  B:0088H.6       PUBLIC        TR1
  B:0090H.3       PUBLIC        RDB
  B:00C8H.2       PUBLIC        TR2
  B:00B8H.0       PUBLIC        PX0
  B:00B8H.2       PUBLIC        PX1
BL51 BANKED LINKER/LOCATER V4.13                                                      04/17/2013  16:59:47  PAGE 41


  B:00B0H.5       PUBLIC        DIN
  C:3555H         PUBLIC        AD7843
  B:00C8H.3       PUBLIC        EXEN2
  B:0090H.0       PUBLIC        TFT_CS
  B:0098H.4       PUBLIC        REN
  D:00C8H         PUBLIC        T2CON
  B:00B0H.3       PUBLIC        KEY
  B:0090H.4       PUBLIC        RES
  B:0090H.2       PUBLIC        WRB
  C:3228H         PUBLIC        Makpix
  B:00B0H.0       PUBLIC        RXD
  B:00B0H.1       PUBLIC        TXD
  C:3727H         PUBLIC        _delay
  B:00B0H.3       PUBLIC        Penirq
  C:3447H         PUBLIC        Getpix
  C:290DH         PUBLIC        _LCD_SetPos
  B:00D0H.5       PUBLIC        F0
  D:00D0H         PUBLIC        PSW
  -------         PROC          SPISTART
  C:373BH         LINE#         7
  C:373BH         LINE#         8
  C:373BH         LINE#         9
  C:373DH         LINE#         10
  C:373FH         LINE#         11
  C:3741H         LINE#         12
  C:3743H         LINE#         13
  -------         ENDPROC       SPISTART
  -------         PROC          _WRITECHARTO7843
  D:0007H         SYMBOL        num
  -------         DO            num
  D:0006H         SYMBOL        count
  -------         ENDDO         count
  C:36B6H         LINE#         18
  C:36B6H         LINE#         19
  C:36B6H         LINE#         20
  C:36B8H         LINE#         21
  C:36BAH         LINE#         22
  C:36BAH         LINE#         23
  C:36BAH         LINE#         24
  C:36BEH         LINE#         25
  C:36C0H         LINE#         26
  C:36C5H         LINE#         27
  C:36CAH         LINE#         28
  C:36CEH         LINE#         29
  -------         ENDPROC       _WRITECHARTO7843
  -------         PROC          READFROMCHARFROM7843
  -------         DO            READFROMCHARFROM7843
  D:0005H         SYMBOL        count
  D:0002H         SYMBOL        Num
  -------         ENDDO         Num
  C:35F2H         LINE#         34
  C:35F2H         LINE#         35
  C:35F2H         LINE#         36
  C:35F4H         LINE#         37
  C:35F6H         LINE#         38
  C:35F6H         LINE#         39
  C:35FDH         LINE#         40
BL51 BANKED LINKER/LOCATER V4.13                                                      04/17/2013  16:59:47  PAGE 42


  C:3602H         LINE#         41
  C:3607H         LINE#         42
  C:3613H         LINE#         43
  C:3617H         LINE#         44
  -------         ENDPROC       READFROMCHARFROM7843
  -------         PROC          _LCD_SETPOS
  D:0014H         SYMBOL        x0
  D:0016H         SYMBOL        x1
  D:0018H         SYMBOL        y0
  D:001AH         SYMBOL        y1
  C:290DH         LINE#         51
  C:2919H         LINE#         52
  C:2919H         LINE#         53
  C:2924H         LINE#         54
  C:292FH         LINE#         55
  C:293AH         LINE#         56
  C:2945H         LINE#         58
  C:294FH         LINE#         59
  C:294FH         LINE#         60
  C:295AH         LINE#         61
  C:2965H         LINE#         62
  C:296CH         LINE#         63
  C:2974H         LINE#         64
  C:2974H         LINE#         65
  C:2980H         LINE#         66
  C:298BH         LINE#         67
  C:2997H         LINE#         68
  C:29A2H         LINE#         69
  C:29AEH         LINE#         70
  C:29B9H         LINE#         71
  C:29C5H         LINE#         72
  C:29D0H         LINE#         73
  C:29D7H         LINE#         74
  C:29D7H         LINE#         75
  C:29DFH         LINE#         76
  C:29DFH         LINE#         77
  C:29EBH         LINE#         78
  C:29F6H         LINE#         79
  C:2A02H         LINE#         80
  C:2A0DH         LINE#         81
  C:2A19H         LINE#         82
  C:2A24H         LINE#         83
  C:2A30H         LINE#         84
  C:2A3BH         LINE#         85
  C:2A42H         LINE#         86
  C:2A42H         LINE#         87
  C:2A4EH         LINE#         88
  C:2A4EH         LINE#         89
  C:2A54H         LINE#         90
  C:2A5CH         LINE#         91
  C:2A63H         LINE#         93
  C:2A6AH         LINE#         94
  C:2A72H         LINE#         95
  C:2A79H         LINE#         97
  C:2A80H         LINE#         98
  C:2A80H         LINE#         99
  C:2A8CH         LINE#         100
BL51 BANKED LINKER/LOCATER V4.13                                                      04/17/2013  16:59:47  PAGE 43


  C:2A8CH         LINE#         101
  C:2A92H         LINE#         102
  C:2A9AH         LINE#         103
  C:2AA1H         LINE#         105
  C:2AA8H         LINE#         106
  C:2AB0H         LINE#         107
  C:2AB7H         LINE#         109
  C:2ABEH         LINE#         110
  C:2ABEH         LINE#         112
  C:2ABEH         LINE#         113
  C:2AC9H         LINE#         114
  C:2AD4H         LINE#         115
  C:2ADBH         LINE#         116
  C:2ADBH         LINE#         118
  -------         ENDPROC       _LCD_SETPOS
  -------         PROC          _DRAWPOINT
  D:0001H         SYMBOL        x
  D:0010H         SYMBOL        y
  D:0012H         SYMBOL        color
  C:34D4H         LINE#         124
  C:34DEH         LINE#         125
  C:34DEH         LINE#         126
  C:34F9H         LINE#         127
  C:3500H         LINE#         128
  C:3507H         LINE#         129
  C:350EH         LINE#         130
  -------         ENDPROC       _DRAWPOINT
  -------         PROC          MAKPIX
  D:0018H         SYMBOL        pix1
  D:001CH         SYMBOL        pix2
  -------         DO            pix2
  D:0005H         SYMBOL        l
  D:0006H         SYMBOL        x
  D:0002H         SYMBOL        y
  -------         ENDDO         y
  C:3228H         LINE#         136
  C:3228H         LINE#         137
  C:3228H         LINE#         138
  C:322AH         LINE#         139
  C:324CH         LINE#         140
  C:326EH         LINE#         141
  C:3284H         LINE#         142
  C:3284H         LINE#         143
  C:3286H         LINE#         144
  C:3297H         LINE#         145
  C:32A8H         LINE#         146
  C:32A8H         LINE#         147
  C:32AAH         LINE#         148
  -------         ENDPROC       MAKPIX
  -------         PROC          AD7843
  -------         DO            AD7843
  D:0018H         SYMBOL        pix
  -------         ENDDO         pix
  C:3555H         LINE#         153
  C:3555H         LINE#         154
  C:3555H         LINE#         156
  C:3557H         LINE#         157
BL51 BANKED LINKER/LOCATER V4.13                                                      04/17/2013  16:59:47  PAGE 44


  C:355CH         LINE#         158
  C:3562H         LINE#         159
  C:3568H         LINE#         160
  C:356FH         LINE#         161
  C:3574H         LINE#         162
  C:357AH         LINE#         163
  C:3580H         LINE#         164
  C:3587H         LINE#         165
  C:3589H         LINE#         167
  C:358FH         LINE#         168
  -------         ENDPROC       AD7843
  -------         PROC          GETPIX
  -------         DO            GETPIX
  D:0010H         SYMBOL        pix1
  D:0014H         SYMBOL        pix2
  -------         ENDDO         pix2
  C:3447H         LINE#         173
  C:3447H         LINE#         174
  C:3447H         LINE#         177
  C:3457H         LINE#         178
  C:3467H         LINE#         180
  C:3490H         LINE#         181
  -------         ENDPROC       GETPIX
  -------         PROC          _DELAY
  D:0006H         SYMBOL        i
  C:3727H         LINE#         186
  C:3727H         LINE#         187
  C:3727H         LINE#         188
  C:3731H         LINE#         189
  -------         ENDPROC       _DELAY
  -------         PROC          INRT
  -------         DO            INRT
  D:0008H         SYMBOL        X
  D:000AH         SYMBOL        Y
  -------         ENDDO         Y
  C:32ABH         LINE#         194
  C:32BEH         LINE#         196
  C:32CAH         LINE#         197
  C:32D1H         LINE#         198
  C:32D4H         LINE#         200
  C:32DBH         LINE#         201
  C:32E0H         LINE#         203
  C:32E7H         LINE#         204
  C:32EDH         LINE#         205
  C:32F3H         LINE#         206
  C:32FAH         LINE#         207
  C:32FFH         LINE#         208
  C:3305H         LINE#         209
  C:330BH         LINE#         210
  C:3312H         LINE#         211
  -------         ENDPROC       INRT
  -------         ENDMOD        TOUCH

  -------         MODULE        ?C?COPY
  C:2BACH         PUBLIC        ?C?COPY
  -------         ENDMOD        ?C?COPY

BL51 BANKED LINKER/LOCATER V4.13                                                      04/17/2013  16:59:47  PAGE 45


  -------         MODULE        ?C?UIDIV
  C:2BD2H         PUBLIC        ?C?UIDIV
  -------         ENDMOD        ?C?UIDIV

LINK/LOCATE RUN COMPLETE.  0 WARNING(S),  0 ERROR(S)
